:020000040800F2
:1000000000000220258200085F0600086106000843
:100010006306000865060008670600080000000087
:100020000000000000000000000000006906000859
:100030006B060008000000006D0600086F0600084F
:10004000758200087706000875820008758200082E
:100050007F06000887060008758200087582000880
:100060007582000875820008758200087582000894
:100070007582000875820008758200087582000884
:100080007582000875820008758200087582000874
:100090007582000875820008758200087582000864
:1000A0007582000875820008758200087582000854
:1000B0007582000875820008758200087582000844
:1000C0007582000875820008758200087582000834
:1000D000758200088906000875820008758200088C
:1000E0007582000875820008000000007582000813
:1000F0007582000875820008758200087582000804
:1001000075820008758200087582000875820008F3
:1001100075820008758200087582000875820008E3
:1001200075820008758200087582000875820008D3
:1001300075820008758200087582000875820008C3
:1001400000000000000000000000000000000000AF
:1001500075820008758200087582000875820008A3
:100160007582000875820008758200087582000893
:100170007582000875820008758200087582000883
:1001800075820008990600087582000875820008CB
:100190007582000875820008758200087582000863
:1001A0007582000875820008758200087582000853
:1001B0009D06000875820008758200087582000897
:1001C0007582000875820008AD060008BD060008AB
:1001D00075820008CD060008758200087582000847
:1001E0007582000875820008758200087582000813
:1001F0007582000875820008758200087582000803
:1002000075820008758200087582000875820008F2
:1002100075820008758200087582000875820008E2
:1002200075820008758200087582000800000000D1
:1002300075820008DD0600080000000075820008D5
:1002400075820008758200087582000875820008B2
:1002500075820008758200087582000875820008A2
:100260007582000875820008758200087582000892
:100270007582000875820008758200080000000081
:100280007582000875820008758200080000000071
:08029000000000007582000867
:1002980053B94AB9002908BF00281CBF4FF0FF31E5
:1002A8004FF0FF3000F00CB8ADF1080C6DE904CE4A
:1002B80008F0F0F8DDF804E0DDE9022304B0704747
:1002C800704700BF10B5054C237833B9044B13B100
:1002D8000448AFF300800123237010BD44010020BF
:1002E800000000004887000808B5034B1BB103490C
:1002F8000348AFF3008008BD00000000480100205B
:100308004887000870B58CB00024079408940994B5
:100318000A940B94314BD3F8E02042F01002C3F852
:10032800E020D3F8E02002F010020192019AD3F8FD
:10033800E02042F00402C3F8E020D3F8E02002F005
:1003480004020292029AD3F8E02042F08002C3F835
:10035800E020D3F8E02002F080020392039AD3F859
:10036800E02042F00102C3F8E020D3F8E02002F0D8
:1003780001020492049AD3F8E02042F00202C3F882
:10038800E020D3F8E02002F002020592059AD3F8A3
:10039800E02042F00802C3F8E020D3F8E03003F090
:1003A80008030693069B0E4D22460221284605F0B7
:1003B80034F90823079308940126099607A90948E0
:1003C80005F026F802230793089609940A9407A9CA
:1003D800284605F01DF80CB070BD00BF0044025857
:1003E800000002580010025808B50A480A4B03607A
:1003F80002234360042383600023C3601822026140
:100408004FF40072426101228261C361036205F008
:10041800EDFF08BD640100200050005238B5104CB3
:10042800104B23604FF4612363600025A560E560ED
:1004380025610C236361A561E56125626562A5629A
:10044800204606F0A8FD2946204606F031FE29463A
:10045800204606F052FE204606F00BFE38BD00BFCF
:10046800B00100200010014070B5CCB04C22002132
:1004780039A807F031FF2022002131A807F02CFF0E
:10048800BC22002102A807F027FF022005F034FA59
:1004980000230193294BDA6A22F00102DA62DB6A4F
:1004A80003F001030193264B9A6942F440429A6192
:1004B8009B6903F440430193019B214B9B6913F40F
:1004C800005FFAD0232339934FF480333A93012203
:1004D8003C9240253D953F92022342934393449397
:1004E80028214591469347924892082649964A936F
:1004F80000244B9439A803F05DF93F23319303237B
:10050800329333943496359536954FF48063379308
:100518003895214631A803F06DFD0A4B029330232C
:100528001493169420944FF4401323930DEB060074
:1005380003F0FCFF05F00AFA4CB070BD0004005847
:10054800004802580100048230B595B005F0CCFA95
:10055800FFF78AFFFFF7D6FEFFF746FFFFF75EFFBC
:1005680001F06EFB344B1B7803B1FEE74FF4807348
:100578000C934FF440630D934FF4005309934FF0DD
:1005880040730F934FF440430E9300240A94FF23C3
:100598000893119412941394EB23069304230B935A
:1005A80001940094254D029502238DF80C308DF8A6
:1005B8000D40214602A800F0CCF902A800F02CFB5F
:1005C8009DF814101E4801F009FB214602A800F00E
:1005D80036FA4FF440730C93012102A800F0B9F9E0
:1005E8000B942246214602A800F0D0F96A4606A9D3
:1005F800284605F066FD00B1B7E7124801F0EEFAAB
:100608004FF0104001F000FB88B90F4801F0E6FAFE
:100618004FF0104001F000FB044601460B4801F082
:10062800DDFA4FF01041204601F000FBE4E70848EE
:1006380001F0D4FAE0E700BF600100206401002067
:10064800688700087C87000890870008A48700084E
:10065800B887000870477047FEE7FEE7FEE7FEE749
:1006680070477047704708B505F06CFA08BD08B5C3
:1006780005F076F908BD08B504F038FE08BD7047E6
:1006880008B5024805F028FF08BD00BFB0010020EA
:100698007047000008B5024805F086FD08BD00BF98
:1006A8006401002008B5024801F080FF08BD00BFC2
:1006B8001C07002008B5024801F078FF08BD00BFFC
:1006C8001C07002008B5024801F070FF08BD00BFF4
:1006D8001C07002008B504F0B1FF08BD00B583B0C1
:1006E8001B4BD3F8F42042F00202C3F8F420D3F8ED
:1006F800F43003F002030193019B0022114601200C
:1007080005F072F9012005F0A5F900221146042030
:1007180005F06AF9042005F09DF90022114605202C
:1007280005F062F9052005F095F9002211465120DF
:1007380005F05AF9512005F08DF9002211467D2067
:1007480005F052F97D2005F085F903B05DF804FB4A
:1007580000440258F0B58BB0002305930693079325
:10076800089309930268354B9A4201D00BB0F0BD4B
:10077800334BD3F8D42042F48042C3F8D420D3F8C2
:10078800D42002F480420192019AD3F8E02042F08A
:100798001002C3F8E020D3F8E02002F01002029221
:1007A800029AD3F8E02042F00202C3F8E020D3F81E
:1007B800E02002F002020392039AD3F8E02042F00C
:1007C8000802C3F8E020D3F8E03003F008030493EC
:1007D800049B04240594022506950926099605A973
:1007E800184804F015FE059406950024079408940B
:1007F8000996154F05A9384604F00AFE4FF46053D0
:100808000593069507940894099605A90F4804F0DE
:10081800FFFD402305930695079408940A2309933E
:1008280005A9384604F0F4FD224601215C2005F0B4
:10083800DBF85C2005F00EF998E700BF0050005285
:10084800004402580010025800040258000C0258D4
:1008580000B589B000230393049305930693079387
:10086800026803F1804303F588339A4202D009B045
:100878005DF804FB164BD3F8F02042F01002C3F8E1
:10088800F020D3F8F02002F010020192019AD3F878
:10089800E02042F00102C3F8E020D3F8E03003F092
:1008A80001030293029B4FF4C06303930223049352
:1008B8000723079303A9074804F0AAFD0022012192
:1008C800252005F091F8252005F0C4F8CFE700BFF2
:1008D80000440258000002584FF480738B610023D3
:1008E8000B62CB620B634B634379012B04D04FF44B
:1008F8000053CB60002070474FF44053CB60F9E7BA
:10090800F0B58FB004460E4617461D466946FFF7F8
:10091800E3FF032300934FF48063079301964FF09E
:1009280080730993002305930A954FF47A726946F8
:10093800206805F048FA10B101200FB0F0BD4FF45F
:100948007A723946206805F0F6FA0028F5D00120B9
:10095800F3E730B58FB004460D466946FFF7BCFF94
:1009680075B1382300930023079309930A930593DD
:100978004FF47A726946206805F025FA0FB030BD49
:100988004FF440730693FF230093ECE710B590B043
:100998000446090101F0300102F0030211438DF809
:1009A8003F1001A9FFF798FF4FF440730793C02346
:1009B8000193002308934FF040720A9201220B9290
:1009C80006934FF47A7201A9206805F0FCF910B17A
:1009D800012010B010BD4FF47A720DF13F0120686C
:1009E80005F040FAF5E730B58FB005466946FFF7E0
:1009F80073FF062300930024079409940A9405942E
:100A08004FF47A726946286805F0DDF920460FB080
:100A180030BD30B58FB005466946FFF75DFF5023FE
:100A280000930024079409940A9405944FF47A7269
:100A38006946286805F0C7F920460FB030BD30B5C3
:100A480091B004460D4602A9FFF746FF35230293ED
:100A5800002309934FF080720B9201220C920793A6
:100A68004FF47A7202A9206805F0ADF910B101209F
:100A780011B030BD4FF47A720DF10701206805F00E
:100A88005AFA18BB9DB12046FFF7ADFF31230293F8
:100A98009DF8073043F002038DF807304FF47A725F
:100AA80002A9206805F08FF928B10120E0E7204667
:100AB800FFF7AFFFEAE74FF47A720DF107012068FC
:100AC80005F0D0F90028D3D00120D1E70120CFE7E5
:100AD80070B594B0054600240E9401260F96129422
:100AE8001196102310934FF4800313936946FFF770
:100AF800F3FE4FF0807309930594052300930A963B
:100B080007940EAA6946286805F084FA08B914B053
:100B180070BD3046FBE770B58EB004460E46694698
:100B2800FFF7DAFE202300934FF480630793002534
:100B380009950A95059501962046FFF754FF4FF44D
:100B48007A726946206805F03EF92046FFF7C0FF33
:100B580028460EB070BD70B58EB004460D461646D8
:100B68006946FFF7B9FE022300934FF480630793A9
:100B78004FF080730993002305934FF480730A9311
:100B880001952046FFF72FFF4FF47A7269462068D7
:100B980005F019F918B1012528460EB070BD4FF4BB
:100BA8007A723146206805F05DF9054608B10125DD
:100BB800F2E72046FFF78CFFEEE710B590B0044649
:100BC80002A9FFF789FE002309934FF080720B9268
:100BD80007939F23029303230C934FF47A7202A97D
:100BE800206805F0F0F810B1012010B010BD4FF4E6
:100BF8007A7201A9206805F09EF958B99DF8043069
:100C080023739DF8053063739DF8062001239340F4
:100C1800A360EAE70120E8E708B5FFF7CEFF08BDC3
:100C280000B583B08DF807004FF47A7301220DF1F7
:100C38000701034806F009F903B05DF804FB00BF9B
:100C4800B001002070470146002007E000EB80005B
:100C5800531C0B60137803EB400030380A68137894
:100C6800303BDBB2092BF1D970472DE9F04F83B047
:100C780005460E4693461F46DDF830A00D9CDDF86C
:100C880038900F9B13F0030F19D1A0460192C84565
:100C980009D202F1010B3B4631462020A84708F152
:100CA80001085A46F3E7DDF804B008E0013C02F118
:100CB80001083B4631461AF80400A8474246002C72
:100CC800F4D10F9B13F0020F03D1104603B0BDE817
:100CD800F08FA2EB0B034B45F7D2541C3B46314631
:100CE8002020A8472246F4E72DE9F04385B09E4628
:100CF8000C9D0D9C9DF83890DDF83C80DDF840C0D7
:100D0800119B129E16F0020F20D16BB116F0010F45
:100D18000AD0B9F1000F02D116F00C0F04D0013B34
:100D280002E030272F5501341F2C98BF6445F8D3B3
:100D380016F0010F0AD01F2C8CBF002701279C42F8
:100D480004D21FB130272F550134F1E716F0100FE8
:100D580027D016F4806F11D184B19C4218BF644526
:100D68000CD1B4F1010C14BF01270027B8F1100F02
:100D780014BF002707F001072FB3023CB8F1100F8A
:100D880023D0B8F1100F29D01F2C98BFB8F1020F4B
:100D980002D162272F5501341F2C02D830272F5536
:100DA80001341F2C05D8B9F1000F20D02D272F555D
:100DB800013403960293019400957346FFF755FF9B
:100DC80005B0BDE8F0836446D8E716F0200FD8D107
:100DD8001F2CD6D878272F550134DDE716F0200FC1
:100DE800D2D01F2CD0D858272F550134D4E716F06D
:100DF800040F03D02B272F550134DAE716F0080F1C
:100E0800D7D020272F550134D3E72DE9F04190B0F2
:100E1800169C189D1B9E0CB926F0100616F4806EC1
:100E28001AD084B34FF0000E16E00CF1300C5FFAC4
:100E38008CFC0EF101070DF14008C6440EF820CCD9
:100E4800B4FBF5FCAC4234BF002401241F2F88BF3B
:100E58000024CCB1BE466446B4FBF5FC05FB1C4C33
:100E68005FFA8CFCBCF1090FDFD916F0200F08D00F
:100E78004127BC445FFA8CFCACF10A0C5FFA8CFC8D
:100E8800D7E76127F5E7274606961A9C0594199C2B
:100E9800049403959DF85C400294019708AC009473
:100EA800FFF722FF10B0BDE8F0812DE9F04F95B0B3
:100EB80009900A910B929B461E9D1F9E229FDDF86A
:100EC8008C80DDF898A055EA060301D12AF0100AB3
:100ED8001AF4806423D055EA060334D000241EE0B7
:100EE80003F13002D2B204F1010914AB1C4404F836
:100EF800202C3A46434628463146FFF7C9F9BD42F9
:100F080076EB08032CBF01230023B9F11F0F8CBF18
:100F1800002303F00103C3B14C4605460E463A468A
:100F2800434628463146FFF7B3F9D3B2092BD7D940
:100F38001AF0200F05D041221A44D2B20A3AD2B28E
:100F4800D1E76122F8E74FF00009CDF818A0259BFA
:100F58000593249B049303979DF880300293CDF862
:100F680004900CAB00935B460B9A0A990998FFF71B
:100F7800BBFE15B0BDE8F08F2DE9F04F89B00446EF
:100F88000D4617461E461299DDF84CA0DDF8509024
:100F9800B4EE400BF1EE10FA40F0AC809FED967B7A
:100FA800B4EEC70BF1EE10FA00F3A4809FED947B2A
:100FB800B4EEC70BF1EE10FA00F19C80B5EEC00B51
:100FC800F1EE10FA00F1A480B0EE405B19F48060F5
:100FD80000D1062115EE902AC2F30A53A3F2FF337B
:100FE80007EE103AC2F3130E15EE102A4EF07F5397
:100FF80043F44013B8EEC77B9FED834B9FED846BA2
:1010080007EE046BB7EE087B43EC142B34EE477BFA
:101018009FED814B07EE046BFDEEC67B17EE908AC1
:10102800B8EEE74B9FED7E6BB6EE007B04EE067BD9
:10103800FDEEC76BB8EEE67B9FED7B3B27EE037BAF
:101048009FED7B3B14EE037B27EE074B16EE903AA1
:1010580003F2FF334FF0000B4FEA035C37EE073B18
:10106800B0EE006B36EE477BB2EE0C6B84EE062BCF
:10107800B2EE046B32EE062B84EE026BB1EE082B57
:1010880036EE026B84EE062B37EE027B83EE076B9F
:10109800B7EE007B36EE077B4CEC16BB27EE067BE3
:1010A800B0EE476BB4EEC57BF1EE10FA05DD08F142
:1010B800FF38B2EE044B87EE046B08F16303C62BCE
:1010C80029D84FF0040B19F4006F2DD09FED5A7BEF
:1010D800B4EEC75BF1EE10FA2BDB9FED597BB4EE53
:1010E800C75BF1EE10FA24D5414517DDA1EB0801E5
:1010F800013914E0CDF80890CDF804A000913346EA
:101108003A462946204600F09FF809B0BDE8F08F1E
:10111800B1EE405B5AE74FF0050BD4E7002149F4E4
:1011280080694FF0000BD846D34508D2AAEB0B03D1
:1011380006E00029F8D00028F6D00139F4E70023AA
:1011480019F00202079203D0BBF1000F00D0002370
:10115800B8F1000F01D085EE065BB5EEC00BF1EEDD
:1011680010FA37D429F40062029201930091B0EE8C
:10117800450B33463A462946204600F065F8BBF150
:10118800000FC2D019F0200F27D04FF0450C00F106
:1011980001093346024629466046A04788EAE872B4
:1011A800A2EBE872052305930BF1FF3304930023A8
:1011B80003930A2302934FEAD873019300923346AC
:1011C8004A4629462046FFF720FE079B002B9CD065
:1011D80002460CE0B1EE455BC4E74FF0650CD6E77C
:1011E80002F10108334629462020A0474246D31B76
:1011F8005345F5D3104688E7FFFFFFFFFFFFEF7F5A
:10120800FFFFFFFFFFFFEFFFFB799F501344D33F22
:10121800B3C8608B288AC63F61436F63A787D23FF4
:1012280071A379094F930A40EF39FAFE422EE63F3F
:101238001655B5BBB16B02402D431CEBE2361A3F85
:101248000000000080842E412DE9F04F8FB0189DDA
:10125800199F1A9EB4EE400BF1EE10FA28D19FEDBB
:10126800AC7BB4EEC70BF1EE10FA2AD49FEDAA7B43
:10127800B4EEC70BF1EE10FA2CDC9FEDA97BB4EEAF
:10128800C70BF1EE10FA36DC9FEDA77BB4EEC70B67
:10129800F1EE10FA2FD4B5EEC00BF1EE10FA30D4FF
:1012A8000024059416F4806F00F08B80002438E049
:1012B80003960297032401949F4C0094FFF7D5FCF2
:1012C800F9E003960297042401949C4C0094FFF7DC
:1012D800CCFCF0E016F0040509D0994C4DB104257A
:1012E8000396029701950094FFF7BFFCE3E0954C45
:1012F800F4E70325F4E7029601970095FFF73CFE13
:10130800D9E09FED8B7B37EE400B01240594C9E7AC
:101318000DF1380CA4444FF030080CF8208C013D36
:1013280001341F2C8CBF4FF0000C4FF0010C092D1D
:1013380098BF4FF0000CBCF1000FE9D1FDEEC07B67
:1013480017EE908AB8EEE77B30EE477BDFF8FCC1FA
:101358000CEBC50C9CED006B27EE067BFCEEC75B27
:1013680015EE909AB8EE655B37EE457BB6EE005BFE
:10137800B4EEC57BF1EE10FA25DD09F1010907EE9F
:10138800909AB8EE677BB4EEC76BF1EE10FA03D80B
:1013980008F101084FF000092DBB07EE908AB8EE5E
:1013A800E77B30EE470BB6EE007BB4EEC70BF1EEF1
:1013B80010FA00D54BDD18F0010F48D008F10108EC
:1013C80045E0062572E7B6EE006BB4EEC67BF1EE9B
:1013D80010FAE1D4B9F1000F02D019F0010FDBD0F7
:1013E80009F10109D8E71F2C22D8013DDFF860C1B7
:1013F800ACFB09EC4FEADC0CE3460CEB8C0CA9EBDC
:101408004C0C04F1010A0CF1300C0DF1380E744447
:1014180004F820CCB9F1090F34D9D9465446E2E78B
:101428000EAD25444FF0300905F8209C654601347F
:101438001F2C03D805F1FF3C002DF1D11F2C06D835
:101448000EAD25444FF02E0C05F820CC01341F2C8E
:101458001BD83D4D85FB08C54FEAE87CCCEBA50CB5
:1014680065460CEB8C0CA8EB4C0C04F101090CF153
:10147800300C0DF13808444404F820CCA8461DB1BE
:101488004C46E4E75446D3E74C4606F00305012DE5
:1014980014D01F2C08D8059D25B30EAD25444FF058
:1014A8002D0C05F820CC013403960297019406AC64
:1014B8000094FFF7DAFB0FB0BDE8F08F6FB1059D20
:1014C80015B916F00C0F08D0013F06E00EAD254403
:1014D8004FF0300C05F820CC01341F2C98BFBC42CB
:1014E800F4D3D6E716F0040F07D00EAD25444FF01D
:1014F8002B0C05F820CC0134D6E716F0080FD3D012
:101508000EAD25444FF0200C05F820CC0134CBE774
:10151800FFFFFFFFFFFFEFFFFFFFFFFFFFFFEF7F73
:101528000000000065CDCD410000000065CDCDC1B3
:101538000000000000000000DC870008E0870008C9
:10154800D4870008D087000867666666E8870008C1
:10155800CDCCCCCC2DE9F04F8FB0074616460D9375
:101568008846002900F0228300240D9B1878002863
:1015780000F01E83252809D0651C334622464146C3
:10158800B8470D9B01330D932C46EEE701330D93BD
:1015980000250D9B1978A1F12002102A0AD8DFE84E
:1015A80002F03809093D0909090909090933092E11
:1015B80009092900A1F13003DBB2092B33D92A2903
:1015C80036D000230A930D9B1A782E2A40D04FF06C
:1015D800000B0D9A1378683B122B77D8DFE803F0DD
:1015E8006476D3765676767676767676727676766C
:1015F8007676D80045F0010501330D93C9E745F02B
:10160800020501330D93C4E745F0040501330D933A
:10161800BFE745F0080501330D93BAE745F010051B
:1016280001330D93B5E70DA8FFF70DFB0A90CAE744
:10163800189B1A1D18921868002804DB0A900D9B45
:1016480001330D93BFE745F0020543420A93F6E7DD
:1016580045F480655A1C0D925A78A2F13003DBB22A
:10166800092B04D92A2A07D04FF0000BB1E70DA89F
:10167800FFF7E9FA8346ACE7189B1A1D18921B6816
:1016880023EAE37B0D9B01330D93A2E745F48071B8
:10169800531C0D9352786C2A01D00D4616E045F480
:1016A800407501330D9311E045F08001531C0D93F3
:1016B8005278682A01D00D4608E045F0C00501338C
:1016C8000D9303E045F4807501320D920D9B187857
:1016D800A0F12503532B00F25F82DFE813F05202DA
:1016E8005D025D025D025D025D025D025D025D02FA
:1016F8005D025D025D025D025D025D025D025D02EA
:101708005D025D025D025D025D025D025D025D02D9
:101718005D025D025D025D025D025D025D026D01BA
:101728004F016D015D025D025D025D025D025D02B9
:101738005D025D025D025D025D025D025D025D02A9
:101748005D025D025E005D025D025D025D025D029A
:101758005D025D025D025D025E0099015E006D0141
:101768004F016D015D025E005D025D025D025D027A
:101778005D025E0037025D025D02D2015D025E001D
:101788005D025D025E0045F4007501320D929DE731
:1017980045F4807501320D9298E7582818BF7828CB
:1017A80007D06F283CD062283CD025F010050A23CA
:1017B80000E01023582837D0692818BF642801D0C2
:1017C80025F00C0515F4806F01D025F0010564287B
:1017D80018BF692876D115F4007F28D115F4807FC9
:1017E80049D115F0400F5FD0189A111D1891127841
:1017F80082EAE271A1EBE27105950A980490CDF8AE
:101808000CB00293D20F0192009133462246414612
:101818003846FFF7FAFA04460D9B01330D93A4E608
:101828000823C7E70223C5E745F02005C4E7189A4F
:10183800073222F0070202F1080118915168126874
:101848000846002913DB08950A9D0795CDF818B0BE
:10185800049300230593C90F029100920190334627
:10186800224641463846FFF720FB0446D4E7524259
:1018780061EB4100E7E7189A111D1891126882EA96
:10188800E271A1EBE27105950A980490CDF80CB0CD
:101898000293D20F019200913346224641463846C0
:1018A800FFF7B3FA0446B7E715F0800F05D0189A8A
:1018B800111D1891B2F900209AE7189A111D189174
:1018C800126895E715F4007F1AD115F4807F33D19B
:1018D80015F0400F45D0189A111D189112780595EA
:1018E8000A990491CDF80CB0029300230193009259
:1018F8003346224641463846FFF787FA04468BE7C7
:10190800189A073222F0070202F108011891089587
:101918000A990791CDF818B0002104930591029116
:10192800D2E90023CDE90023334622464146384612
:10193800FFF7BBFA04466FE7189A111D1891059531
:101948000A990491CDF80CB002930023019313680F
:1019580000933346224641463846FFF756FA044676
:101968005AE715F0800F04D0189A111D18911288A3
:10197800B5E7189A111D18911268B0E7462818D0D3
:10198800189B073323F0070303F10802189293ED1D
:10199800000B02950A9B0193CDF800B0334622460E
:1019A80041463846FFF750FC04460D9B01330D9322
:1019B800DBE545F02005E3E7472814BF00230123B2
:1019C800672814BF1A4643F001020AB145F40065BE
:1019D800452808BF43F001030BB145F02005189BCB
:1019E800073323F0070303F10802189293ED000B65
:1019F80002950A9B0193CDF800B033462246414632
:101A08003846FFF7B9FA04460D9B01330D93ACE550
:101A180015F002051FD04FF001091898031D1893FF
:101A280004F1010A3346224641460078B847BDB959
:101A38000D9B01330D93544697E502F1010A334695
:101A480041462020B8474B46524603F101099B45C1
:101A5800F3D81446E1E70123DDF828B02246F4E77D
:101A68005246DDF828A006E0551C334641462020A2
:101A7800B847A1462A4609F10104CA45F4D8924656
:101A8800D6E7189B1A1D1892D3F800A0BBF1000FD7
:101A98001ED14FF0FF33D14602E009F10109134688
:101AA80099F8002012B15A1E002BF6D1A9EB0A09A9
:101AB80015F480630B9302D0D94528BFD94615F099
:101AC80002030C9306D022465C46B3460B9E1DE0EB
:101AD8005B46E0E722460A9C4B4607E002F1010913
:101AE800334641462020B8472B464A465D1C9C4257
:101AF800F4D8A9465C46B3460B9E07E01C460AF19B
:101B0800010A551C5B464146B8472A469AF8000028
:101B180020B1002EF3D0631E002CEFD114465E4690
:101B28000C9B1BB90D9B01330D931EE5DDF828A016
:101B380006E0551C334641462020B847A1462A46B0
:101B480009F10104CA45F4D81446EBE745F021052C
:101B5800189B1A1D18921B68059508220492CDF847
:101B68000CB01022029200220192009333462246C2
:101B780041463846FFF749F904460D9B01330D935A
:101B8800F3E4651C3346224641462520B8470D9BA1
:101B980001330D932C46E8E4651C33462246414642
:101BA800B8470D9B01330D932C46DEE4074FDBE469
:101BB800B44201D3721E00E022463346414600205B
:101BC800B84720460FB0BDE8F08F00BF4D0C0008A5
:101BD80000B9704708B5FFF723F808BD0FB400B582
:101BE80085B006AA52F8043B039200924FF0FF32E8
:101BF80002A90448FFF7AEFC05B05DF804EB04B099
:101C0800704700BFD91B00080368B3F1804F01D2A9
:101C1800002070470120704740686FF0104303446C
:101C28006FF07042934200D30020704708B572B637
:101C38004FF0E02300221A615A619A61804708BD7B
:101C480008B50821164803F0E1FC012802D1154B1C
:101C58001B78C3B1134B01221A7000221249134892
:101C680005F0AEFA80B91249104805F0C5FA70B906
:101C780010490E4806F0CAFA60B90C4805F0D0FAC7
:101C880058B903F063FE08BDFEF7E4FCEBE7FEF786
:101C9800E1FCEDE7FEF7DEFCEFE7FEF7DBFCF0E743
:101CA8000010025860010020000000203C020020C3
:101CB8007C0000205000002012230B800048704751
:101CC8001C00002004230B800048704730000020CF
:101CD800002393421ED200B510E00CF1370C01F836
:101CE80013C000014FEA430C0CF1010C4FF0000E39
:101CF80001F80CE00133DBB2934209D24FEA107CC1
:101D0800B0F1204FE9D20CF1300C01F813C0E8E72C
:101D18005DF804FB7047000038B50B4BD3F800089A
:101D2800D3F80448D3F80838C01800D138BD074D97
:101D38000822A91CFFF7CCFF042205F11201204656
:101D4800FFF7C6FFF2E700BF00E0F11F34000020F4
:101D580008B51A230B80FFF7DFFF014808BD00BF55
:101D68003400002008B50A4628B90549054805F099
:101D7800D6FE034808BD0249024805F0D0FEF8E740
:101D88000C0500203888000810B50A46034C214687
:101D9800034805F0C4FE204610BD00BF0C05002016
:101DA8005888000808B50A4628B90549054805F0C5
:101DB800B6FE034808BD0249024805F0B0FEF8E740
:101DC8000C0500206C88000808B50A4628B90549A2
:101DD800054805F0A4FE034808BD0249024805F07D
:101DE8009EFEF8E70C050020788800080020704760
:101DF80041B1012904D1002393700A215170137055
:101E08000020704700239370642151701370F7E726
:101E180070B504460D4616460221084803F003FC37
:101E280021460748FFF7DAFE33462A4604F1E04127
:101E38000448FEF765FD002070BD00BF0000025891
:101E4800888800080C0700202DE9F04383B0074676
:101E5800894614460221164803F0E5FB3B780093B7
:101E680023463A4649461348FFF7B8FEC4F3072805
:101E780014F0FF0F03D008F101085FFA88F8002476
:101E88000FE0260209EB042505F1E04529460A483A
:101E9800FFF7A4FEBA1929460848FEF75CFE01348C
:101EA800E4B2A045EDD8002003B0BDE8F08300BF40
:101EB80000000258A8880008EC8800080C070020D9
:101EC80010B5044601460548FFF788FE04F1E041D5
:101ED8000348FEF720FE002010BD00BF0C89000853
:101EE8000C07002038B50A4C0A4B236002232371E3
:101EF8000025657129462046FEF72BFD2046FEF792
:101F08008BFE217B0448FFF769FE284638BD00BFD9
:101F18000C070020640100202C89000830B589B026
:101F28000023039304930593069307930268214BB8
:101F38009A4201D009B030BD1F4CD4F8E03043F0CC
:101F48000103C4F8E030D4F8E03003F00103019352
:101F5800019B4FF4C0530393022504950A2307936A
:101F680003A9164803F054FAD4F8D83043F00063B4
:101F7800C4F8D830D4F8D83003F000630293029B39
:101F880000220121622003F02FFD622003F062FD90
:101F980000220121632003F027FD632003F05AFD8E
:101FA80000222946652003F01FFD652003F052FD3D
:101FB800C0E700BF00000840004402580000025873
:101FC80008B500F57171D0F8040405F050F908BDA2
:101FD80008B5C1EBC10300EB8303D3F80822D0F89E
:101FE800040405F070F908BD08B5C1EBC10300EBA6
:101FF80083039A6CD0F8040405F09EF908BD08B56F
:10200800D0F8040405F034FA08BD10B50446C368D6
:102018003BB1022B01D1012104E0FEF71BFB01219A
:1020280000E00021D4F8040405F00BFAD4F8040405
:1020380005F0DEF910BD000010B50446D0F8040420
:1020480005F002FA2268D2F8003E43F00103C2F814
:10205800003E236A23B1034A136943F00603136160
:1020680010BD00BF00ED00E008B5D0F8040405F08D
:10207800F4F908BD08B5D0F8040405F009FA08BD5C
:1020880008B5D0F8040405F001FA08BD08B5D0F881
:10209800040405F0FFF908BD08B5D0F8040405F0FC
:1020A800FBF908BD02780AB10020704710B5034655
:1020B8001548C0F80434C3F8C402144B036009235C
:1020C80043600222C260002303618261C36103622C
:1020D80043628362C362036300F0E6F880B90A4C86
:1020E8008021204600F01AFE40220021204600F000
:1020F800EFFD80220121204600F0EAFD002010BDFE
:10210800FEF7A8FAEBE700BF1C0700200000084014
:10211800D0F8C43211F0800F08D101F07F01C1EB73
:10212800C10103EB810191F8FE01704701F07F01C5
:10213800C1EBC10103EB810191F83E007047032810
:1021480005D8DFE800F005040205012070470320E8
:10215800704708B5D0F8C40200F044F9FFF7EFFF64
:1021680008BD08B5D0F8C40200F05DF9FFF7E7FF35
:1021780008BD08B594461A466346D0F8C40200F074
:1021880085FCFFF7DCFF08BD08B5D0F8C40200F0F5
:1021980020FDFFF7D4FF08BD08B5D0F8C40200F051
:1021A8005CFDFFF7CCFF08BD08B5D0F8C40200F00D
:1021B80059FCFFF7C4FF08BD08B5D0F8C40200F009
:1021C800D9FCFFF7BCFF08BD08B5D0F8C40200F081
:1021D800A2FCFFF7B4FF08BD2DE9F04383B0D0F8A7
:1021E8000080C1EBC10300EB83035A6D1B6D9A425B
:1021F80054D807460C469B1AC1EBC10200EB820279
:10220800526C9A4200D31A4602F103094FEA99091F
:1022180015E006F103094FEA9909C4EBC40507EB79
:102228008505A96C3B7C0093B3B2E2B2404601F04D
:1022380067F8AB6C3344AB646B6D33446B6508EB88
:10224800441303F510639B699BB24B4512D3C4EB4F
:10225800C40207EB8202516D136D99420AD24BB149
:102268005B1AC4EBC40207EB8202566C9E42D0D3C1
:102278001E46CEE7C4EBC40007EB80073A6D7B6DC2
:102288009A420FD804F00F040123A340D8F8344829
:1022980024EA0304C8F83448002000E0012003B011
:1022A800BDE8F0830020FAE770B58AB0002800F096
:1022B80097800546046890F8BD333BB3032385F83F
:1022C800BD33E36B13F4807F01D100232B612868B1
:1022D80000F01AFE2C4654F8106BEC460FCCACE814
:1022E8000F000FCCACE80F0094E803008CE8030063
:1022F8002B1D0ECB304600F049FD044658B1022391
:1023080085F8BD33012420460AB070BD80F8BC337F
:10231800FFF704FED2E70021286800F0FBFD234602
:1023280016E0C3EBC30205EB8202012182F83D10DF
:1023380082F83C30A2F84230002182F83F10516404
:102348009164C3EBC30205EB820211650133DBB272
:1023580069688B42E5D316E0C4EBC40305EB83033D
:10236800002283F8FD2183F8FC4183F8FF21C3F89C
:102378000422C3F80822C4EBC40305EB8303C3F8A3
:1023880010220134E4B2A142E6D82C4654F8106B6E
:10239800EC460FCCACE80F000FCCACE80F0094E88B
:1023A80003008CE803002B1D0ECB304600F0F8FD2F
:1023B800044660B9002385F83830012385F8BD3319
:1023C8006B6A012B08D0286801F072F99BE7022399
:1023D80085F8BD33012496E7284600F0A3FCF2E710
:1023E800012490E7026890F8BC33012B19D010B58E
:1023F8000446012380F8BC33836A012B09D0206886
:1024080001F04AF9206800F079FD002084F8BC0347
:1024180010BD8369012BF2D0936B43F4803393632F
:10242800EDE70220704738B590F8BC33012B18D07F
:102438000446012380F8BC33006800F065FD20687D
:1024480001F0FAF8054628B1002384F8BC330125C9
:10245800284638BD206801F02BF9002384F8BC33E6
:10246800F6E70225F4E7000070B504460D4600685B
:10247800066C00EB411303F530639A682169012962
:1024880011D034498E424ED03DB9C5EBC50304EB9B
:102498008303D3F81032002B56D0E9B22046FFF759
:1024A80097FD002070BD12F0080F09D02A498E420E
:1024B800F7D912F4004FF4D04FF400429A60F0E7D5
:1024C80012F0200F02D020229A60EAE712F0280FBB
:1024D800E7D121498E4206D912F4004F03D04FF4B8
:1024E80000429A60DDE7C5EBC50204EB8202D2F830
:1024F80004121B69C3F31203CB1AC2F81432D2F8C0
:1025080008320B44C2F8083215B9D2F8103223B198
:10251800E9B22046FFF75CFDC3E704F571720121BB
:1025280001F018F9F4E712F4004F03D04FF4004219
:102538009A60B6E712F0200F01D020229A60E9B223
:102548002046FFF745FDACE704F57172002101F064
:1025580001F9A2E70A31544F0A30544F38B50446FE
:1025680003681D6C03EB4113D3F8081B0E4A954210
:1025780007D903F5306311F4004F02D04FF400423D
:102588009A602046FFF71CFD074B9D4202D923693C
:10259800012B01D0002038BD04F57172012120689B
:1025A80001F0D8F8F6E700BF0A30544F2DE9F84F8C
:1025B80004460568284601F0B8F808B1BDE8F88F68
:1025C8000646206801F080F80028F7D0206801F05E
:1025D8007BF810F0020F04D02268536903F002035D
:1025E8005361206801F070F810F0100F14D02268C1
:1025F800936923F0100393612F6A07F00F08C7F35C
:102608004343022B00F08580062B00F0A18022684E
:10261800936943F010039361206801F055F810F4B2
:10262800002F40F0A780206801F04EF810F4802FAA
:1026380040F0E980206801F047F80028C0F2538193
:10264800206801F041F810F4006F0AD0D5F8083876
:1026580013F0010F40F061812268536903F40063AD
:102668005361206801F030F810F0006F15D022682F
:10267800536903F00063536194F8F433002B40F07E
:102688005081012184F8F41323685B6DC3F383033D
:10269800C4F8F833204600F059FB206801F014F81C
:1026A80010F4805F40F04181206801F00DF810F4CB
:1026B800005F40F09581206801F006F810F0080FDF
:1026C80040F0A681206800F0FFFF10F4801F40F062
:1026D800A881206800F0F8FF10F4001F40F0AB81DB
:1026E800206800F0F1FF10F0804F40F0AE812068C4
:1026F80000F0EAFF10F0040F3FF460AF23685D6854
:1027080015F0040F40F0AA81226853682B435360E8
:1027180054E747F6F0731F423FF479AF4FEA171BAF
:10272800C8EBC80904EB8909C7F30A12D9F80812DB
:10273800284600F017FFCBF30A02D9F808321344F1
:10274800C9F80832D9F814321A44C9F814225EE7D5
:10275800082204F57171284600F004FFC7F30A1730
:10276800C8EBC80204EB8202D2F814321F44C2F844
:1027780014724CE7206800F0ABFF0746B04616E03D
:1027880005EB48130122C3F8082B41462046FFF702
:102798006BFE1BE005EB48130822C3F8082B4146E3
:1027A8002046FFF7DBFE14E008F101087F08002F40
:1027B8003FF439AF17F0010FF6D05FFA88F12068BF
:1027C80000F096FF814610F0010FD9D119F0080FDB
:1027D800E0D119F0100F04D005EB48131022C3F80C
:1027E800082B19F0200F04D005EB48132022C3F85A
:1027F800082B19F4005FD7D005EB48134FF40052AB
:10280800C3F8082BD0E7206800F06AFF0746B046F7
:1028180029E051462046FFF7E7FB19F0080F04D0DE
:1028280005EB48130822C3F8082919F0100F04D043
:1028380005EB48131022C3F8082919F0400F04D0FB
:1028480005EB48134022C3F8082919F0020F04D0F9
:1028580005EB48130222C3F8082919F0800F3DD16F
:1028680008F101087F08002F3FF4E4AE17F0010FCC
:10287800F6D05FFA88FA5146206800F042FF814698
:1028880010F0010FC9D008F00F03012101FA03F27B
:10289800D5F8343823EA0203C5F8343805EB481371
:1028A800C3F8081923698B42B3D1C8EBC80304EBFA
:1028B8008303596C9A6C0A449A64B8F1000FA8D142
:1028C800C8EBC80304EB83031B6D002BA1D104F5EF
:1028D80071720121206800F03DFF9AE741462046C9
:1028E800FFF77AFCBCE7D5F8043823F00103C5F8F4
:1028F800043894F8F433012B08D02046FFF7B4FBD2
:102908002268536903F00043536199E6002184F873
:10291800F413204600F01AFAF2E72046FFF78CFB82
:102928009AE62046FFF788FBB7E605F500677B685F
:1029380023F001037B601021206800F003FB20E0F6
:1029480005EB46134FF67F31C3F80819D3F8002971
:1029580022F40012C3F80029D3F8002942F00062DB
:10296800C3F80029C3F8081BD3F8002B22F400127F
:10297800C3F8002BD3F8002B42F00062C3F8002BF9
:1029880001366368B342DBD8FB6943F00113FB618E
:10299800236BDBB1D7F8843043F00B03C7F88430DE
:1029A8007B6C43F00B037B64D5F8003823F4FE639B
:1029B800C5F8003804F57172217C206800F0CAFE61
:1029C8002268536903F4805353616DE67A6942F2D1
:1029D8002B0313437B613B6943F00B033B61E3E744
:1029E800206800F0A7FE206800F09EFBE0602568E4
:1029F80001F04AFC0146227B284600F00DFA2046E9
:102A0800FFF703FB2268536903F40053536152E64E
:102A18002046FFF7F4FA2268536903F0080353616C
:102A280050E600212046FFF72BFB2268536903F488
:102A3800801353614DE600212046FFF71BFB2268F7
:102A4800536903F4001353614AE62046FFF71EFB5F
:102A58002268536903F08043536148E62046FFF734
:102A68001BFB51E690F8BC33012B0DD010B5044682
:102A7800012380F8BC3380F83810006800F0FCFDB2
:102A8800002084F8BC0310BD0220704738B5054605
:102A98008C4611F0800F29D101F00F0ECEEBCE0439
:102AA800A40004F5FC740444211DCEEBCE0E00EB0B
:102AB8008E0E00208EF8FD010CF00F0C81F800C07E
:102AC8008A60CB704A780AB1A1F806C0022B1DD0E3
:102AD80095F8BC33012B1CD0012385F8BC3328683A
:102AE80000F032FB002085F8BC0338BD01F00F0070
:102AF800C0EBC0018900383129440431C0EBC00063
:102B080005EB8000012480F83D40D5E700230B71D8
:102B1800DEE70220E9E710B501F00F04C4EBC401B9
:102B2800890001F5FC7101440431C4EBC40C00EBCD
:102B38008C0CCCF80822CCF810320023CCF81432D4
:102B48008CF8FD318CF8FC410369012B06D064B97F
:102B5800DAB2006800F046FB002010BDC4EBC40CDC
:102B680000EB8C0CCCF80C22F1E7DAB2006800F02C
:102B7800DFFBF1E710B501F00F04C4EBC4018900D5
:102B8800383101440431C4EBC40C00EB8C0CCCF894
:102B98004820CCF850300023CCF8543001238CF86E
:102BA8003D308CF83C400369012B06D064B9DAB299
:102BB800006800F017FB002010BDC4EBC40C00EB4C
:102BC8008C0CCCF84C20F1E7DAB2006800F0B0FBCE
:102BD800F1E738B501F00F054268954239D8044647
:102BE8000B4611F0800F1FD1C1EBC101890001F51F
:102BF800FC7101440431C3EBC30300EB83030022DF
:102C080083F8FD2101238B700D7094F8BC33012BE0
:102C180021D0012384F8BC33206800F0B2FC8DB1C8
:102C2800002084F8BC0338BDC5EBC50189003831E4
:102C380001440431C5EBC50300EB8303012283F88B
:102C48003D20DFE704F57172217C206800F082FDE9
:102C5800E6E70120E7E70220E5E701F00F03426815
:102C6800934231D810B5044611F0800F1ED1C3EB42
:102C7800C301890001F5FC7101440431C3EBC302AF
:102C880000EB8202002082F8FD0100228A700B709E
:102C980094F8BC33012B19D0012384F8BC33206885
:102CA80000F09CFC002084F8BC0310BDC3EBC301FA
:102CB8008900383101440431C3EBC30200EB8202BE
:102CC800012082F83D00E0E7012070470220ECE790
:102CD80010B40468606A31B940EA0240A06200207A
:102CE8005DF8044B70478C46A36A00EB1340002341
:102CF80008E003F1400104EB8101496800EB114051
:102D08000133DBB20CF1FF318B42F2D340EA0240CF
:102D18000CF13F0104EB81014860E0E70368596268
:102D280000207047034602680121C0F8FC13002008
:102D380083F8F403936943F000639361516D024B88
:102D48000B435365704700BF030000107047000035
:102D5800002301330C4A934211D80269002AF8DA99
:102D6800036943F00103036100230133064A9342D8
:102D780007D8026912F0010FF7D10020704703202D
:102D880070470320704700BF400D030084B010B5A2
:102D9800044603A880E80E00089B012B1DD1A36BF5
:102DA80023F48033A363E2681A4B1340E360E368BB
:102DB80023F44013E3600F9B012B09D02046FFF753
:102DC800C7FF069B012B1BD0BDE8104004B070471D
:102DD800E36843F48013E360F0E7E36843F04003FB
:102DE800E3602046FFF7B4FF0C9B23B9A36B43F4C1
:102DF8008033A363E5E7A36B23F48033A363E0E7A1
:102E0800A36843F00603A360A36843F02003A3600C
:102E1800DAE700BFBFFFBDFF022A0AD00921C26856
:102E280022F47052C260C36843EA8123C360002061
:102E38007047204B0B44204A934229D91F4B0B441F
:102E48001F4A934226D91F4B0B441F4A934223D94A
:102E58001E4B0B441E4A934220D31E4B0B441E4A62
:102E680093421DD91D4B0B441D4A93421AD31D4B47
:102E78000B441D4A934217D31C4B0B441C4A9342E4
:102E880014D31C4B0B441C4A934211D20721C6E7AA
:102E98000F21C4E70E21C2E70D21C0E70C21BEE7D0
:102EA8000B21BCE70A21BAE70921B8E70821B6E7F0
:102EB8000621B4E7405327FFFF340C00401E1BFFD8
:102EC8003F420F0000DC0BFF7F4F1200808CF9FEA1
:102ED80020D6130060B6E5FE5FE3160000D3CEFEF1
:102EE80040771B00C05BB3FEC091210000CA91FE71
:102EF80020753800E05459FEE09C4100836843F097
:102F08000103836000207047836823F00103836016
:102F18000020704708B5C36823F0C043C360012987
:102F280009D069B9C36843F08043C360322002F016
:102F38001BFE002008BDC36843F00053C360F5E7DB
:102F48000120F7E7890141F02001016100230133E5
:102F5800054A934205D8026912F0200FF7D10020E4
:102F680070470320704700BF400D03001023036122
:102F780000230133054A934205D8026912F0100F65
:102F8800F7D1002070470320704700BF400D0300B1
:102F9800D0F800381943C0F8001800207047000026
:102FA80084B02DE9F041044607A880E80E0000230C
:102FB80006E003F1400204EB820200215160013374
:102FC8000E2BF6D9119F27BBD4F8043843F002031F
:102FD800C4F80438A36B23F40013A363236843F0F5
:102FE80040032360236843F0800323600023C4F870
:102FF800003E04F50065D4F80038C4F800380C9B8E
:10300800012B10D1099B4BB900212046FFF7C0FFC7
:103018000DE0A36B43F40013A363E7E70121204607
:10302800FFF7B6FF03E003212046FFF7B1FF1021A9
:103038002046FFF787FF804608B14FF00108204679
:10304800FFF794FF08B14FF0010800232B616B6173
:10305800EB610AE0C3B94FF00060C2F80009002232
:103068000A614FF67F328A6001330799994210D975
:1030780004EB431202F51061D2F800090028E9DBDD
:103088000020C2F80009EAE74FF09040C2F80009B2
:10309800E5E700230AE0C3B14FF0904CC2F800CB3B
:1030A800002202614FF67F3282600133994211D9C2
:1030B80004EB431202F53060D2F8006B002EEADB15
:1030C8004FF0000CC2F800CBEAE74FF0006CC2F8F2
:1030D80000CBE5E72B6923F480732B610023A36100
:1030E8006FF0804363610A9B1BB9A36943F0100327
:1030F800A361A2690A4B1343A3610D9B1BB1A3698A
:1031080043F00803A361012F04D04046BDE8F04115
:1031180004B07047A269034B1343A361F5E700BFEE
:1031280000383C8004000040D0F8083813F006034B
:1031380005D0062B18BF022B03D1022070470020B0
:1031480070470F207047000010B591F800C04B7809
:10315800012B21D000F5006ED0F81C380CF00F04BC
:103168000122A24043EA0243C0F81C3800EB4C108D
:10317800D0F8003B13F4004F0CD1D0F8002B8B682B
:10318800C3F30A03C97843EA81431343144A1A4331
:10319800C0F8002B002010BDD0F81C280CF00F0E32
:1031A80003FA0EF39BB21343C0F81C3800EB4C1023
:1031B800D0F8003913F4004FECD1D0F800298B680F
:1031C800C3F30A03C97843EA814343EA8C5C42EAC1
:1031D8000C0C034B4CEA0303C0F80039DAE700BFD4
:1031E8000080001070B40B784C78012C25D000EBCF
:1031F800431000F530631D693F4C2C401C611D696C
:103208003E4C2C401C614C690CB18C684C611C69AB
:1032180044F400241C611C698D68C5F3120C44EA4F
:103228000C041C61012A62D0D0F8003B43F004432F
:10323800C0F8003B002070BC70474C695CBB00EBD9
:103248004314D4F810692D4D3540C4F81059D4F8FA
:10325800105945F40025C4F81059D4F81069264DC2
:103268003540C4F81059012A32D000EB4313D3F883
:10327800002942F00442C3F800294B69002BD9D039
:10328800D0F834380A7802F00F0101228A4013433B
:10329800C0F83438CEE700EB431404F5106426690F
:1032A800154D354025612669144D354025618D68D9
:1032B8004E69AE4200D94D61256945F40025256166
:1032C80025694E69C6F3120C45EA0C052561CAE763
:1032D8000A691AB100EB4311C1F8142900EB431035
:1032E800D0F8002942F00442C0F80029A2E7CA68D1
:1032F800002A99D05A6197E70000F8FFFFFF07E01E
:1033080010B59DF8084084B903334FEA930E4FF087
:10331800000C08E000EB023303F5805351F8044B2E
:103328001C600CF1010CF445F4D3002010BD000022
:10333800F0B583B00B784C78012C31D000EB4313F7
:1033480003F5306CDCF81050834C2C40CCF810405E
:10335800DCF81050814C2C40CCF810404C69002C03
:1033680040F0C680DCF810408D68C5F312052C4388
:10337800CCF81040DCF8104044F40024CCF810409D
:10338800012A00F0CF80CA78012A00F0D280D3F851
:10339800002B42F00442C3F8002B002003B0F0BD1C
:1033A8004C6974BB00EB4314D4F810696B4D35407D
:1033B800C4F81059D4F8105945F40025C4F8105928
:1033C800D4F81069644D3540C4F81059012A4DD01D
:1033D80000EB4313D3F8004944F00444C3F8004910
:1033E800CC78012C6BD04B69002BD6D0D0F8343870
:1033F8000A7802F00F0101228A401343C0F83438DA
:10340800CBE700EB4314D4F81069534D3540C4F8AA
:103418001059D4F81069514D3540C4F81059D4F8F2
:1034280010598E684F6907EB060C0CF1FF3CBCFB8A
:10343800F6FC4B4E06EACC4C45EA0C05C4F810598C
:10344800D4F810594E69C6F312063543C4F810591A
:1034580004F51064CD78012DB8D1256925F0C04553
:103468002561256945F000552561AFE70A691AB15C
:1034780000EB4314C4F81429CA78012A08D000EBD9
:103488004313D3F8002942F00442C3F8002984E723
:10349800D0F8082812F4807F08D100EB4311D1F846
:1034A800002942F00052C1F80029E8E700EB431177
:1034B800D1F8002942F08052C1F80029DFE7D0F89E
:1034C800084814F4807F0CD1D3F8004944F0005424
:1034D800C3F8004900928B8A0A78C968FFF710FF81
:1034E8005BE7D3F8004944F08054C3F80049F1E79A
:1034F8008D682C44013CB4FBF5F4DCF810501FFA3D
:1035080084FE174E06EAC4442543CCF81050DCF874
:1035180010508C680EFB04F4C4F312042C43CCF84E
:1035280010402DE7CA68002A3FF42DAFCCF81420CC
:1035380029E7D0F8082812F4807F06D1D3F8002BA9
:1035480042F00052C3F8002B21E7D3F8002B42F0D9
:103558008052C3F8002B1AE70000F8FFFFFF07E0CE
:103568000000F81F84460846D11C8908002305E09E
:103578000CF58052126840F8042B01338B42F7D3C4
:1035880070470B784A78012A14D000EB4310D0F822
:10359800002B002A06DB2BB1D0F8003B23F0804338
:1035A800C0F8003BD0F8003B43F40013C0F8003BE0
:1035B8000020704700EB4310D0F80029002A06DBF2
:1035C8002BB1D0F8003923F08043C0F80039D0F887
:1035D800003943F40013C0F80039E9E70B784A785A
:1035E800012A0ED000EB4310D0F8003B23F400135F
:1035F800C0F8003BCB78023BDBB2012B15D9002089
:10360800704700EB4310D0F8003923F40013C0F8DA
:103618000039CB78023BDBB2012BF0D8D0F8003967
:1036280043F08053C0F80039E9E7D0F8003B43F095
:103638008053C0F8003BE2E710B50446002208E0DA
:1036480004EB42134FF67F31C3F80819C3F8081B7F
:1036580001320E2AF4D90022C4F81028C4F814281C
:10366800C4F81C282046FFF781FC00B110BD1021CA
:103678002046FFF767FCF9E7D0F8003823F4FE632B
:10368800C0F80038D0F80038090101F4FE61194388
:10369800C0F800180020704708B5D0F8043823F0A7
:1036A8000203C0F80438032002F05EFA002008BDC7
:1036B80008B5D0F8043843F00203C0F804380320F2
:1036C80002F052FA002008BD426980691040704734
:1036D800D0F8183800F50060C0691840000C704731
:1036E800D0F8183800F50060C069184080B27047FB
:1036F80000EB4111D1F8082B00F50060406910403B
:10370800704710B4D0F81048D0F8343801F00F02E0
:10371800D340DB01DBB2234300EB411000F510601E
:10372800806818405DF8044B7047406900F001005C
:1037380070470000D0F80029054B1340C0F8003945
:10374800D0F8043843F48073C0F804380020704778
:1037580000F8FFFF10B4046C154B9C4203D9D0F855
:10376800003B002B16DB0024C0F8104BD0F8104BA0
:1037780044F40024C0F8104BD0F8104B44F018045F
:10378800C0F8104BD0F8104B44F0C044C0F8104BB0
:10379800012903D000205DF8044B7047C0F8142BB2
:1037A800D0F8003B43F08023C0F8003BF2E700BFAD
:1037B8000A30544F002800F0048338B504460368E3
:1037C80013F0010F25D09D4A136903F03803926A5C
:1037D800102B15D0182B0FD06368B3F5803F3FD05E
:1037E800002B54D1954B1A6822F480321A601A685B
:1037F80022F480221A6038E002F00302022AEBD198
:103808008E4B1B6813F4003F03D06368002B00F055
:10381800DA82236813F0020F00F08D80874A13695B
:10382800926A13F038035CD0182B57D0E368002B4A
:1038380000F0CA8081490A6822F0190213430B601C
:1038480002F08CF905467D4B1B6813F0040F40F01D
:10385800998002F083F9401B0228F4D90320B9E2C9
:10386800764A136843F480331360636833B302F015
:1038780075F90546714B1B6813F4003FC9D102F076
:103888006DF9401BB0F57A7FF4D90320A2E2B3F5B5
:10389800A02F09D0694B1A6822F480321A601A687E
:1038A80022F480221A60E0E7644B1A6842F480220E
:1038B8001A601A6842F480321A60D6E702F04EF9AC
:1038C80005465E4B1B6813F4003FA2D002F046F990
:1038D800401BB0F57A7FF4D903207BE212F0030F86
:1038E800A4D1564B1B6813F0040F03D0E368002BD8
:1038F80000F06B8202F04CF941F20303984212D8AF
:103908002269402A07D04D494B6823F47C3343EAA7
:1039180002334B600FE0494A536823F47C3343F485
:103928000033536007E0454A536823F0FE4321699A
:1039380043EA01635360236813F0100F00F0888096
:103948003E4A136903F03803926A082B54D0182BA7
:103958004ED0E369002B00F0B880384A136843F072
:103968008003136002F0FAF80546344B1B6813F421
:10397800807F40F0888002F0F1F8401B0228F4D9DB
:10398800032027E202F004F941F20303984212D817
:103998002269402A07D029494B6823F47C3343EA3B
:1039A80002334B60C7E7254A536823F47C3343F45A
:1039B80000335360BFE7214A536823F0FE4321696F
:1039C80043EA01635360B6E71C4A136823F0010316
:1039D800136002F0C3F80546184B1B6813F0040F78
:1039E800A9D002F0BBF8401B0228F5D90320F1E169
:1039F80002F00302012AACD1104B1B6813F4807F3C
:103A080003D0E369802B40F0E28102F0C1F841F273
:103A18000303984214D8226A202A07D007494B6822
:103A280023F0F84343EA82634B6011E0034A53688A
:103A380023F0F84343F08043536009E00044025800
:103A48009A4AD36823F07C53216A43EA0163D3601E
:103A5800236813F0080F60D06369002B49D0934A9C
:103A6800536F43F00103536702F078F805468F4B14
:103A78005B6F13F0020F50D102F070F8401B022860
:103A8800F5D90320A6E102F083F841F20303984236
:103A980012D8226A202A07D084494B6823F0F843B9
:103AA80043EA82634B60D3E7804A536823F0F843C4
:103AB80043F080435360CBE77C4AD36823F07C53C0
:103AC800216A43EA0163D360C2E7784A136823F0A6
:103AD8008003136002F042F80546744B1B6813F428
:103AE800807FB5D002F03AF8401B0228F5D90320B0
:103AF80070E16E4A536F23F00103536702F02EF80A
:103B080005466A4B5B6F13F0020F06D002F026F8E9
:103B1800401B0228F5D903205CE1236813F0200F2D
:103B280029D0A3699BB1614A136843F48053136099
:103B380002F014F805465D4B1B6813F4005F1AD1B8
:103B480002F00CF8401B0228F5D9032042E1574A3D
:103B5800136823F48053136002F000F80546534BB2
:103B68001B6813F4005F06D001F0F8FF401B022821
:103B7800F5D903202EE1236813F0040F21D1636ADD
:103B8800002B00F02681494A126902F03802182AEF
:103B980000F0EE80022B75D0444A136823F080733E
:103BA800136001F0DBFF0446404B1B6813F0007FF5
:103BB80000F0DC8001F0D2FF001B0228F4D90320BA
:103BC80008E13B4A136843F48073136001F0C6FFB1
:103BD8000546374B1B6813F4807F06D101F0BEFF02
:103BE800401B6428F5D90320F4E0A368012B0AD010
:103BF8000BBB2E4B1A6F22F001021A671A6F22F0C4
:103C080004021A6704E0294A136F43F0010313679B
:103C1800A36833B301F0A2FF0546244B1B6F13F0D2
:103C2800020FACD101F09AFF401B41F28833984251
:103C3800F3D90320CEE0052B09D01C4B1A6F22F0D4
:103C480001021A671A6F22F004021A67E0E7174B9D
:103C58001A6F42F004021A671A6F42F001021A67DB
:103C6800D6E701F07BFF0546104B1B6F13F0020FE0
:103C780085D001F073FF401B41F288339842F3D995
:103C88000320A7E0094A136823F08073136001F04A
:103C980065FF0546054B1B6813F0007F0AD001F04D
:103CA8005DFF401B0228F5D9032093E00044025829
:103CB800004802584F4B996A4F4A0A40A16AE06A85
:103CC80041EA00110A439A62226B013AC2F30802E0
:103CD800616B0139490289B20A43A16B01390904B0
:103CE80001F4FE010A43E16B0139090601F0FE41C6
:103CF8000A431A63DA6A22F00102DA62596B3F4A10
:103D08000A40A16C42EAC1025A63DA6A22F00C0244
:103D1800216C0A43DA62DA6A22F00202616C0A4311
:103D2800DA62DA6A42F48032DA62DA6A42F400323B
:103D3800DA62DA6A42F48022DA62DA6A42F001026E
:103D4800DA621A6842F080721A6001F007FF0446CE
:103D5800284B1B6813F0007F06D101F0FFFE001B03
:103D68000228F5D9032035E0002033E0002031E0B7
:103D7800204A916A106B012B2DD001F00303A26A2F
:103D880093422AD1C1F30511E36A994227D1C0F3BE
:103D98000802236B013B9A4223D1C0F34622636B8E
:103DA800013B9A421FD1C0F30642A36B013B9A42E2
:103DB8001BD1C0F30660E36B013B984217D100208A
:103DC80008E001207047012004E0012002E0012002
:103DD80000E0002038BD0120FCE70120FAE70120BF
:103DE800F8E70120F6E70120F4E70120F2E70120D7
:103DF800F0E700BF004402580CFCFFFF0700FFFF7C
:103E0800744B1B6903F03803102B00F0DE80182B6D
:103E180010D00BB1704870476E4B1B6813F0200F21
:103E280000F0D5806B4B1868C0F3C1006B4B23FAC8
:103E380000F0704710B4674A916A01F00301946A70
:103E4800C4F30510D36A03F0010C536BC3F3CC031E
:103E58000CFB03F307EE903AF8EE677A14F47C7FD4
:103E680000F09380012965D0022900F09180E1B12A
:103E780007EE100AF8EE476A9FED596A86EE267A31
:103E8800544B1B6BC3F3080306EE903AF8EE666AD0
:103E98009FED546A67EE867A76EEA77AF7EE006AA7
:103EA80077EEA67A27EE277A60E0136813F0200FE2
:103EB80023D011461268C2F3C102484BD34007EE23
:103EC800103AF8EE476A07EE100AB8EE476A86EE2F
:103ED800867A0B6BC3F3080306EE903AF8EE666A2F
:103EE8009FED406A67EE867A76EEA77AF7EE006A6B
:103EF80077EEA67A27EE277A38E007EE100AF8EE72
:103F0800476A9FED396A86EE267A324B1B6BC3F3FC
:103F1800080306EE903AF8EE666A9FED326A67EE9D
:103F2800867A76EEA77AF7EE006A77EEA67A27EE1B
:103F3800277A1BE007EE100AF8EE476A9FED286A19
:103F480086EE267A234B1B6BC3F3080306EE903AE2
:103F5800F8EE666A9FED236A67EE867A76EEA77AB0
:103F6800F7EE006A77EEA67A27EE277A194B1B6BD5
:103F7800C3F34623013307EE903AF8EE677AC7EEAB
:103F8800276AFCEEE67A17EE900A5DF8044B704754
:103F980007EE100AF8EE476A9FED146A86EE267A55
:103FA8000C4B1B6BC3F3080306EE903AF8EE666AF7
:103FB8009FED0C6A67EE867A76EEA77AF7EE006ACE
:103FC80077EEA67A27EE277AD0E7094870470348A4
:103FD800704700BF0044025800093D000090D0031C
:103FE8000024744A000000390024744C0024F44A68
:103FF80000127A00002800F0328170B50D460446A0
:104008009B4B1B6803F00F038B420BD2984A136833
:1040180023F00F030B431360136803F00F038B4265
:1040280040F01F81236813F0040F0CD02269914BD4
:104038009B6903F070039A4205D98E498B6923F076
:1040480070031A438A61236813F0080F0CD0626961
:10405800884BDB6903F070039A4205D98549CB691F
:1040680023F070031A43CA61236813F0100F0CD0B1
:10407800A269804BDB6903F4E0639A4205D97D4964
:10408800CB6923F4E0631A43CA61236813F0200F55
:104098000CD0E269774B1B6A03F070039A4205D98A
:1040A80074490B6A23F070031A430A62236813F0F9
:1040B800020F0CD0E2686F4B9B6903F00F039A4222
:1040C80005D96C498B6923F00F031A438A61236869
:1040D80013F0010F41D0674A936923F47063A16814
:1040E8000B4393616368022B0AD0032B27D0012B63
:1040F8002CD0604A126812F0040F06D10120ADE0FE
:10410800126812F4003F00F0AE805A490A6922F0A2
:10411800070213430B6101F021FD0646554B1B694D
:1041280003F038036268B3EBC20F16D001F016FD36
:10413800801B41F288339842F0D903208EE04D4A23
:10414800126812F0007FE0D1012087E0494A126826
:1041580012F4807FD9D1012080E0236813F0020F88
:104168000CD0E268434B9B6903F00F039A4205D2D7
:1041780040498B6923F00F031A438A613C4B1B6843
:1041880003F00F03AB420AD9394A136823F00F032F
:104198002B431360136803F00F03AB4265D1236808
:1041A80013F0040F0CD02269324B9B6903F07003A3
:1041B8009A4205D22F498B6923F070031A438A610A
:1041C800236813F0080F0CD062692A4BDB6903F0EF
:1041D80070039A4205D22749CB6923F070031A432A
:1041E800CA61236813F0100F0CD0A269214BDB6958
:1041F80003F4E0639A4205D21E49CB6923F4E063D5
:104208001A43CA61236813F0200F0CD0E269194BD6
:104218001B6A03F070039A4205D216490B6A23F011
:1042280070031A430A62FFF7EBFD12498B69C3F367
:104238000323114AD35C03F01F03D8408B6903F0B2
:104248000F03D35C03F01F0320FA03F30B4A136038
:104258000B4B18600B4B186801F01EFC70BD012059
:1042680070470120FAE70120F8E70120F6E700BFD0
:1042780000200052004402588C8900087800002071
:10428800740000207000002008B5FFF7B9FD0B4A44
:104298009369C3F303230A49CB5C03F01F0320FA95
:1042A80003F3926902F00F02885C00F01F0023FA02
:1042B80000F0044A1060044A136008BD0044025824
:1042C8008C890008780000207400002008B5FFF7EA
:1042D800DBFF054BDB69C3F30213044AD35C03F02D
:1042E8001F03D84008BD00BF004402588C8900084D
:1042F80008B5FFF7C9FF054BDB69C3F30223044A7E
:10430800D35C03F01F03D84008BD00BF0044025827
:104318008C890008404B9B6A03F00303032B79D078
:1043280070B505460E463C4A136823F08063136057
:1043380001F014FC0446384B1B6813F0006F06D0DC
:1043480001F00CFC031B022BF5D9032070BD324B86
:104358009A6A22F47C32296842EA01329A626A68CF
:10436800013AC2F30802A9680139490289B20A432D
:10437800E9680139090401F4FE010A432969013990
:10438800090601F0FE410A439A63DA6A22F0C00284
:1043980069690A43DA62DA6A22F02002A9690A43E3
:1043A800DA62DA6A22F01002DA62D96B1B4A0A4032
:1043B800E96942EAC102DA63DA6A42F01002DA62B3
:1043C800C6B91A46DB6A43F40023D362124A13685B
:1043D80043F08063136001F0C1FB04460E4B1B6879
:1043E80013F0006F14D101F0B9FB001B0228F5D9B6
:1043F8000320ABE7012E05D0074AD36A43F4001324
:10440800D362E3E7044AD36A43F48013D362DDE757
:1044180000209BE701207047004402580700FFFF77
:10442800404B9B6A03F00303032B79D070B5054614
:104438000E463C4A136823F08053136001F08EFB4C
:104448000446384B1B6813F0005F06D001F086FB6A
:10445800031B022BF5D9032070BD324B9A6A22F058
:104468007C72296842EA01529A626A68013AC2F388
:104478000802A9680139490289B20A43E968013981
:10448800090401F4FE010A4329690139090601F00A
:10449800FE410A431A64DA6A22F4406269690A43EF
:1044A800DA62DA6A22F40072A9690A43DA62DA6A1D
:1044B80022F48072DA62596C1B4A0A40E96942EABE
:1044C800C1025A64DA6A42F48072DA62C6B91A46DC
:1044D800DB6A43F48003D362124A136843F08053C3
:1044E800136001F03BFB04460E4B1B6813F0005FA2
:1044F80014D101F033FB001B0228F5D90320ABE7E8
:10450800012E05D0074AD36A43F08073D362E3E7EC
:10451800044AD36A43F40003D362DDE700209BE733
:1045280001207047004402580700FFFFF8B5044611
:10453800036813F0006F30D0436EB3F5001F26D028
:104548000ED8EBB1B3F5801F07D102210430FFF775
:10455800E1FE054645B12E4621E0012635461EE01E
:10456800B3F5401F09D10025954A136D23F4401374
:10457800616E0B431365002611E0012635460EE0F7
:104588008F4AD36A43F40033D3620025ECE7022153
:104598002430FFF745FF0546DCE70026354623684B
:1045A80013F4807F14D0636D042B30D8DFE803F058
:1045B800032228080800824AD36A43F40033D362EE
:1045C80045BB7F4A136D23F00703616D0B431365E9
:1045D800236813F4007F2FD0A36D802B49D01ED8F9
:1045E800002B40D0402B17D10021201DFFF792FE51
:1045F800054619E00021201DFFF78CFE0546DFE780
:10460800002104F12400FFF70BFF0546D8E7012637
:104618003546DDE72E46DBE7012635460CE0C02BA4
:1046280002D0B3F5807F1BD155BB654A136D23F4C7
:10463800E073A16D0B431365236813F4806F45D0B5
:10464800D4F8A430B3F5800F38D01ED883B3B3F5AF
:10465800001F17D10021201DFFF75CFE05461AE058
:1046680001263546E8E7564AD36A43F40033D36255
:10467800DAE7002104F12400FFF7D2FE0546D3E76C
:104688002E46D9E70126354620E0B3F5C00F02D003
:10469800B3F5000F09D1C5B9494A936D23F46003F6
:1046A800D4F8A4100B43936510E0012635460DE0BD
:1046B800434AD36A43F40033D362ECE7002104F1A0
:1046C8002400FFF7ADFE0546E5E72E46236813F400
:1046D800006F23D0D4F8A830B3F1007F41D00DD8B3
:1046E800002B38D0B3F1807F05D10021201DFFF7C2
:1046F80011FE054608E0012635460FE0B3F1407F7C
:1047080002D0B3F1806F23D1002D31D12C4A936DA3
:1047180023F0E063D4F8A8100B439365236813F0E3
:10472800007F2ED0A36C202B3FD026D833B1102B7E
:1047380020D1234AD36A43F40033D362002D3AD1FF
:104748001F4AD36C23F03003A16C0B43D36418E0E9
:1047580001263546E2E71A4AD36A43F40033D362A6
:10476800D2E7002104F12400FFF75AFE0546CBE703
:104778002E46D3E70126354603E0302BDED001264E
:104788003546236813F4805F2BD0E36DB3F5005FE3
:104798004CD017D8002B43D0B3F5805F0DD1002142
:1047A800201DFFF7B7FD054612E00221201DFFF787
:1047B800B1FD0546C2E72E46E3E70126354610E07F
:1047C80000440258B3F5405F02D0B3F5804F24D1BE
:1047D800002D32D1754A136D23F4E043E16D0B438C
:1047E8001365236813F4005F37D0236EB3F5003FD9
:1047F80051D027D83BB1B3F5803F20D10121201DEE
:10480800FFF788FD0546002D4CD1684A136D23F447
:10481800E023216E0B4313651FE001263546E0E7D0
:10482800624AD36A43F40033D362D1E7002104F12A
:104838002400FFF7F5FD0546CAE72E46D1E7012615
:1048480035460AE0B3F5802FDDD0B3F5A02FDAD0D6
:10485800B3F5403FD7D001263546236813F4804F7F
:1048680030D0D4F8AC30B3F1005F44D01FD83BB19E
:10487800B3F1805F18D10121201DFFF74BFD0546DC
:10488800002D3FD1494A936D23F0E043D4F8AC1092
:104898000B43936516E0012104F12400FFF7C0FDE6
:1048A8000546B0E72E46D8E7012635460AE0B3F1BB
:1048B800804FE5D0B3F1A04FE2D0B3F1405FDFD035
:1048C80001263546236813F4004F09D0E36EB3F18F
:1048D800805F19D0B3F1005F24D0D3B101263546EB
:1048E800236813F0807F32D0636C032B59D8DFE83C
:1048F80003F026215226012104F12400FFF790FD40
:104908000546BDE72E46DDE7284AD36A43F400335F
:10491800D3626DB9254A136D23F04053E16E0B4302
:104928001365DDE70121201DFFF7F4FC0546F0E7DC
:104938002E46D5E71D4AD36A43F40033D3629DBBA4
:104948001A4AD36C23F00303616C0B43D3642368C6
:1049580013F4800F2CD1236813F0010F00F0A3800B
:10496800A36F282B00F29D80DFE803F08B9B9B9BB5
:104978009B9B9B9B869B9B9B9B9B9B9B949B9B9B9B
:104988009B9B9B9B8B9B9B9B9B9B9B9B8B9B9B9B8F
:104998009B9B9B9B8B000221201DFFF7BBFC0546C0
:1049A800CDE701263546D2E72E46D0E70044025827
:1049B8008F4A136843F48073136001F0CFF80746F9
:1049C8008B4B1B6813F4807F05D101F0C7F8C01B1F
:1049D8006428F5D90325002D4AD1864B1B6FD4F8DE
:1049E800B020534013F4407F0CD0824B1A6F22F44E
:1049F8004072196F41F480311967196F21F48031C1
:104A080019671A67D4F8B030B3F5807F15D08DBB1D
:104A1800D4F8B03003F44072B2F5407F1ED0754A26
:104A2800136923F47C53136172490B6FD4F8B020D7
:104A3800C2F30B0213430B678DE701F08FF80746AB
:104A48006C4B1B6F13F0020FE1D101F087F8C01B0C
:104A580041F288339842F3D90325D8E765480269BB
:104A680022F47C52644901EA131313430361DBE720
:104A78002E4670E72E466EE70121201DFFF74AFCFF
:104A88000546E5B95B4A536D23F03803A16F0B4324
:104A9800536508E0012104F12400FFF7C1FC054635
:104AA800EFE701263546236813F0020F16D0636F2F
:104AB800052B27D8DFE803F00A051F0A0A0A2E4645
:104AC800F1E70121201DFFF725FC0546EDB9494A0C
:104AD800536D23F00703616F0B435365236813F08D
:104AE800040F22D0D4F89030052B43D8DFE803F028
:104AF800140F3B141414012104F12400FFF790FC57
:104B08000546E3E701263546E8E72E46E6E70121B4
:104B1800201DFFF7FFFB05467DBB364A936D23F04A
:104B28000703D4F890100B439365236813F0200F04
:104B380033D0D4F88C30B3F1005F4CD022D83BB1DD
:104B4800B3F1805F1BD10021201DFFF7E3FB054671
:104B5800002D47D1274A536D23F0E043D4F88C1039
:104B68000B43536519E0012104F12400FFF758FCB9
:104B78000546D1E701263546D7E72E46D5E7012673
:104B880035460AE0B3F1804FE2D0B3F1A04FDFD051
:104B9800B3F1405FDCD001263546236813F0400F9F
:104BA80037D0D4F89830B3F5006F52D026D83BB13F
:104BB800B3F5806F18D10021201DFFF7ABFB054628
:104BC800002D4DD10B4A936D23F4E053D4F898107F
:104BD8000B4393651DE0022104F12400FFF720FC3C
:104BE8000546B5E72E46D8E70126354611E000BF51
:104BF8000048025800440258CFFFFF00B3F5805F19
:104C0800DED0B3F5A05FDBD0B3F5406FD8D0012676
:104C18003546236813F0800F32D0D4F89C30B3F5B2
:104C2800804F00F09D8020D83BB1B3F5005F19D1CB
:104C38000021201DFFF76EFB0546002D40F09780F0
:104C4800A34A936D23F46043D4F89C100B439365F7
:104C580016E0022104F12400FFF7E2FB0546AFE766
:104C68002E46D6E7012635460AE0B3F5004FE4D0D4
:104C7800B3F5204FE1D0B3F5C04FDED0012635465D
:104C8800236813F0080F0CD0D4F88030B3F5805F98
:104C98006FD08F4A536D23F44053D4F880100B43E0
:104CA8005365236813F0100F0CD0D4F89430B3F583
:104CB800807F67D0864A936D23F44073D4F89410AC
:104CC8000B439365236813F4002F0BD0D4F8A0305E
:104CD800B3F5803F6ED0B3F5003F61D0002B5AD0BA
:104CE80001263546236813F4802F0CD0D4F884307D
:104CF800B3F5001F76D0B3F5401F69D0B3F5801F18
:104D080061D001263546236813F4803F07D0E36C51
:104D1800002B70D0B3F5803F7BD001263546236841
:104D280013F0005F7DD1236813F4003F00F0868004
:104D3800E36FB3F5807F00F0BA807CD9B3F5007FCC
:104D480003D0B3F5407F40F0B080002D40F0B5802F
:104D58005F4A536D23F44073E16F0B4353656DE075
:104D6800022104F12400FFF75BFB054665E72E46A8
:104D780086E7022104F12400FFF752FB002888D0BF
:104D8800012686E7022104F12400FFF749FB0028E9
:104D980090D001268EE70021201DFFF7BBFA0546BB
:104DA8007DB94B4A936D23F44033D4F8A0100B43DC
:104DB800936597E7022104F12400FFF731FB0546CC
:104DC800EEE72E468EE7424AD36A43F40033D362B5
:104DD8007DB93F4A536D23F44013D4F884100B4334
:104DE800536590E7012104F12400FFF719FB0546FC
:104DF800EEE72E4687E7364AD36A43F40033D36298
:104E08006DB9334AD36C23F48033E16C0B43D3641C
:104E180085E70221201DFFF77DFA0546F0E72E46BB
:104E28007DE7022104F12400FFF7FAFA00283FF495
:104E38007AAF012677E7002B87D00126236813F481
:104E4800801F06D0224A136D23F00043216F0B43C5
:104E58001365236813F0805F07D01D4A136923F494
:104E68008043D4F8B4100B431361236813F4001F74
:104E780006D0174A136D23F08073A16E0B43136598
:104E8800236813F0804F09D0114B1A6922F40042AD
:104E98001A611A69D4F8B8100A431A612368002BFA
:104EA8000DDB06B101263046F8BD0126C6E7084AE3
:104EB800D36A43F40033D36247E72E46BEE7044A79
:104EC800D36C23F04053216D0B43D364E9E700BF53
:104ED8000044025808B5FFF7D7F9054B1B6AC3F31E
:104EE8000213044AD35C03F01F03D84008BD00BF77
:104EF800004402588C89000810B5774A916A946A70
:104F0800C4F3053ED36AC3F3001CD36BC3F3CC03CD
:104F18000CFB03F314F47C3F00F0D88001F003018C
:104F280007EE903AF8EE677A012965D0022900F079
:104F3800B080E1B107EE10EAB8EE477A9FED676AF4
:104F4800C6EE076A644B9B6BC3F3080307EE103A7F
:104F5800B8EE477A9FED626A67EE867A77EE277A2F
:104F6800B7EE007A77EE877A66EEA76A60E0136894
:104F780013F0200F23D011461268C2F3C102594B17
:104F8800D34007EE103AB8EE477A06EE90EAB8EE4C
:104F9800666AC7EE066A8B6BC3F3080307EE103A1E
:104FA800B8EE477A9FED4E6A67EE867A77EE277AF3
:104FB800B7EE007A77EE877A66EEA76A38E007EEF2
:104FC80010EAB8EE477A9FED486AC6EE076A424B88
:104FD8009B6BC3F3080307EE103AB8EE477A9FEDD0
:104FE800406A67EE867A77EE277AB7EE007A77EE30
:104FF800877A66EEA76A1BE007EE10EAB8EE477AF2
:105008009FED366AC6EE076A334B9B6BC3F3080302
:1050180007EE103AB8EE477A9FED316A67EE867A66
:1050280077EE277AB7EE007A77EE877A66EEA76A88
:10503800294A936BC3F3462307EE103AB8EE477A32
:10504800B7EE006A37EE067AC6EE877AFCEEE77AA4
:10505800C0ED007A936BC3F3064307EE103AB8EE3F
:10506800477A37EE067AC6EE877AFCEEE77AC0ED25
:10507800017A936BC3F3066307EE903AF8EE677A0A
:1050880077EE867A86EEA77ABCEEC77A80ED027A4A
:1050980010BD07EE10EAB8EE477A9FED146AC6EE27
:1050A800076A0D4B9B6BC3F3080307EE103AB8EE83
:1050B800477A9FED0B6A67EE867A77EE277AB7EE26
:1050C800007A77EE877A66EEA76AB1E70023036075
:1050D80043608360DCE700BF004402580024744A40
:1050E800000000390090D0030024744C0024F44AD6
:1050F80010B5774A916A946AC4F3055ED36AC3F31C
:10510800002C536CC3F3CC030CFB03F314F07C7F2B
:1051180000F0D88001F0030107EE903AF8EE677AC4
:10512800012965D0022900F0B080E1B107EE10EA4C
:10513800B8EE477A9FED676AC6EE076A644B1B6C48
:10514800C3F3080307EE103AB8EE477A9FED626A98
:1051580067EE867A77EE277AB7EE007A77EE877A67
:1051680066EEA76A60E0136813F0200F23D011469B
:105178001268C2F3C102594BD34007EE103AB8EE99
:10518800477A06EE90EAB8EE666AC7EE066A0B6CD6
:10519800C3F3080307EE103AB8EE477A9FED4E6A5C
:1051A80067EE867A77EE277AB7EE007A77EE877A17
:1051B80066EEA76A38E007EE10EAB8EE477A9FED88
:1051C800486AC6EE076A424B1B6CC3F3080307EE36
:1051D800103AB8EE477A9FED406A67EE867A77EE26
:1051E800277AB7EE007A77EE877A66EEA76A1BE031
:1051F80007EE10EAB8EE477A9FED366AC6EE076A00
:10520800334B1B6CC3F3080307EE103AB8EE477A2A
:105218009FED316A67EE867A77EE277AB7EE007AE5
:1052280077EE877A66EEA76A294A136CC3F346239A
:1052380007EE103AB8EE477AB7EE006A37EE067A0C
:10524800C6EE877AFCEEE77AC0ED007A136CC3F3FA
:10525800064307EE103AB8EE477A37EE067AC6EEFE
:10526800877AFCEEE77AC0ED017A136CC3F3066324
:1052780007EE903AF8EE677A77EE867A86EEA77AA6
:10528800BCEEC77A80ED027A10BD07EE10EAB8EEE0
:10529800477A9FED146AC6EE076A0D4B1B6CC3F381
:1052A800080307EE103AB8EE477A9FED0B6A67EEEF
:1052B800867A77EE277AB7EE007A77EE877A66EE07
:1052C800A76AB1E70023036043608360DCE700BF9F
:1052D800004402580024744A000000390090D003AA
:1052E8000024744C0024F44A7047704710B53D4BB5
:1052F8001B6913F4803F18D03B4B1B78DBB2012BA2
:1053080029D0394B1C78E4B2072C18BF022C47D09F
:10531800032C49D0043CE4B2022C06D9324B0022BB
:105328001A70304B4FF480325A612E4B1B6913F4BC
:10533800DC0348D02C4A91691943916129494B6192
:105348001378DBB2012B34D0072B18BF022B46D0C1
:10535800254B186932E0244B5A68013A5A605B6859
:1053680083B1214CE068FFF7BFFF1E4B4FF480323A
:105378005A61E3680133E360E068A268012100F044
:1053880035F8D2E7184B4FF0FF32DA6000221A7076
:10539800D868FFF7A9FF134B4FF480325A61C4E76E
:1053A8000120FFF7A1FFB5E70F4B1869FFF79CFF36
:1053B800B0E71346D0684FF0FF32DA600A4B00229C
:1053C8001A70FFF792FF084B1B783BB9054AD36860
:1053D80023F4DE03D360044B00221A7510BD0120AC
:1053E800ECE700BF00200052240B002011F0010F51
:1053F8000BD00649CB6823F4E663CB60CB6842EA5E
:1054080000221A4342F08402CA607047002000520A
:10541800F0B583B0002340E0092400E00024B44044
:1054280044EA0C040235764E46F825404FF0B04465
:10543800D4F88050D44325EA02064F6817F4803F19
:1054480001D042EA05064FF0B045C5F88060D5F8AE
:10545800845004EA05064F6817F4003F01D042EA79
:1054680005064FF0B045C5F884602D6804EA0506C6
:105478004F6817F4801F01D042EA05064FF0B04587
:105488002E606D682C404E6816F4001F01D042EA69
:1054980005044FF0B042546001330A6832FA03F44D
:1054A80000F0AB804FF0010C0CFA03FC1CEA02027E
:1054B800F2D04C68651E112C18BF012D01D9122C91
:1054C80013D185685E000324B44025EA0405CC683E
:1054D800B4402C438460446824EA0C0C4C68C4F340
:1054E80000149C4044EA0C044460C6684FEA430C2C
:1054F800032505FA0CF5EC4326EA050E8D6805FA36
:105508000CF545EA0E05C5604D68122D18BF022D31
:1055180012D1DE08083650F8267003F007054FEA66
:10552800850E0F2505FA0EF527EA05070D6905FA18
:105538000EF53D4340F82650056825404C6804F0B8
:10554800030404FA0CF42C4304604C6814F0805FE4
:10555800A2D02C4CD4F8F45045F00205C4F8F4500D
:10556800D4F8F44004F002040194019C9D08AE1C98
:10557800234C54F8267003F00304A6000F24B4400B
:1055880027EA040C204CA0423FF448AF04F580649D
:10559800A04222D004F58064A04220D004F58064A3
:1055A800A0421ED004F58064A0421CD004F580649B
:1055B800A0421AD004F58064A04218D004F5806493
:1055C800A04216D004F58064A04214D004F580648B
:1055D800A0423FF421AF0A2421E701241FE7022457
:1055E8001DE703241BE7042419E7052417E706240D
:1055F80015E7072413E7082411E703B0F0BD00BF3F
:105608000004005800440258000002580369194277
:1056180001D001207047002070470AB181617047AE
:10562800090481617047436931EA030301D081614C
:1056380070470904816170477047000008B5054B41
:10564800D8681A6822EA00021A605860FFF7F4FF67
:1056580008BD00BF00650258002800F0298108B580
:10566800024690F83530DBB2022B03D08023436525
:10567800012008BD0368904890498B4218BF8342B7
:105688000CBF0121002166D03030834263D018302E
:10569800834260D0183083425DD0183083425AD09C
:1056A8001830834257D01830834254D000F55670D2
:1056B800834250D0183083424DD0183083424AD0AC
:1056C8001830834247D01830834244D01830834280
:1056D80041D0183083423ED0183083423BD01968FD
:1056E80021F00E0119601368A0F5956073498B428B
:1056F80018BF83426AD072498B4267D018318B42F7
:1057080064D018318B4261D018318B425ED0183189
:105718008B425BD018318B4258D001F556718B42C1
:1057280054D018318B4251D018318B424ED0183199
:105738008B424BD018318B4248D018318B4245D020
:1057480018318B4242D018318B423FD0196821F072
:10575800010119603EE0042082F8350081BB584AF7
:1057680093422DD0183293422AD01832934227D030
:105778001832934224D01832934221D018329342DF
:105788001ED002F5567293421AD01832934217D09F
:105798001832934214D01832934211D018329342DF
:1057A8000ED0183293420BD01832934208D01832D8
:1057B800934205D01A6822F001021A60002058E7C7
:1057C8001A6822F001021A60002052E7196821F0D5
:1057D800010119601368384838498B4218BF834261
:1057E80042D018318B423FD018318B423CD018310F
:1057F8008B4239D018318B4236D018318B4233D096
:1058080018318B4230D001F556718B422CD01831AB
:105818008B4229D018318B4226D018318B4223D0A5
:1058280018318B4220D018318B421DD018318B4251
:105838001AD018318B4217D022498B4214D0143118
:105848008B4211D014318B420ED014318B420BD0C5
:1058580014318B4208D014318B4205D014318B425D
:1058680002D014318B4217D1116E0B6823F4807368
:105878000B60906DD36D03F01F0101238B404360D3
:10588800536E916E5960D36E33B1196821F48071EB
:105898001960136F516F5960002382F83430012367
:1058A80082F83530136D2BB1104698470020E0E69A
:1058B800012070470020DCE610000240280002406A
:1058C800400002400854025890B190F83D30DBB2D5
:1058D800022B03D08023836601207047042380F8BD
:1058E8003D300268D36823F00103D360002070477D
:1058F8000120704770470000134BDB6813F0040F5A
:1059080007D1114BDB6803F0070383421AD001204B
:10591800704710B50C4AD36823F007031843D060CA
:1059280000F01CF90446084B5B6813F4005F07D1CC
:1059380000F014F9001BB0F57A7FF4D9012000E0DB
:10594800002010BD0020704700480258024AD36862
:1059580043F08073D36070470048025870470000D6
:1059680008B5174B1B6813F0100F06D04FF0B04363
:10597800D3F8883013F4803F0CD1114B1B6813F413
:10598800803F06D04FF0B043D3F8883013F4803FFF
:105998000BD108BDFFF7AEFF4FF0B042D2F8883008
:1059A80043F48033C2F88830E7E7FFF7D7FF4FF0BA
:1059B800B042D2F8883043F48033C2F88830E8E740
:1059C800004802580649CB6823F4E0631B041B0C0B
:1059D800000200F4E0600343024A1A43CA607047B9
:1059E80000ED00E00000FA0500B5174BDB68C3F3D3
:1059F8000223C3F1070CBCF1040F28BF4FF0040CBD
:105A080003F1040EBEF1060F14D9033B4FF0FF3E1D
:105A18000EFA0CFC21EA0C0199400EFA03F322EA73
:105A280003031943002807DB0901C9B2074B1954BE
:105A38005DF804FB0023E9E700F00F000901C9B293
:105A4800034B1954F4E700BF00ED00E000E400E068
:105A580014ED00E0002807DB00F01F0240090123D5
:105A68009340024A42F82030704700BF00E100E04E
:105A78000138B0F1807F0BD24FF0E0235861054A1E
:105A8800F02182F823100020986107221A617047DC
:105A98000120704700ED00E0104B1B780BB9012086
:105AA800704710B504464FF47A70B0FBF3F30C4A14
:105AB8001068B0FBF3F0FFF7DBFF68B90F2C01D9D2
:105AC80001200AE0002221464FF0FF30FFF78CFF4B
:105AD800044B1C60002000E0012010BD6C00002079
:105AE800740000207000002010B50320FFF76AFF43
:105AF800FEF786F90F498B69C3F303230E4AD35C7B
:105B080003F01F03D8408B6903F00F03D35C03F045
:105B18001F0320FA03F3094A1360094B1860002099
:105B2800FFF7BAFF10B10124204610BD0446FAF76A
:105B3800D5FDF9E7004402588C8900087800002058
:105B480074000020034B1B78034A11680B44136050
:105B5800704700BF6C000020400B0020014B186804
:105B6800704700BF400B002038B50446FFF7F6FF2A
:105B78000546B4F1FF3F02D0044B1B781C44FFF7E5
:105B8800EDFF401BA042FAD338BD00BF6C000020D7
:105B9800014B1868000C70470010005CF0B44B6AA9
:105BA80033B1B2F1406F03D08B6A0468013B2361C3
:105BB8008C69002C6ED00E6A002E3BD003688C686E
:105BC800DC61CC69F4B1CB6A0D6B2B434D6B2B4375
:105BD8004D6A2B434D6943EA85430D692B430D6A92
:105BE8002B43CD682B4323438C6923430C68234301
:105BF800046813436361B2F1406F19D003684A68BF
:105C08009A6115E0CB6A0D6B2B434D6B2B434D6AA4
:105C18002B434D6943EA85430D692B430D6A2B439A
:105C280023438C6923430C68234301681A434A6160
:105C3800F0BC7047CD69D5B1CB6A0F6B3B434F6B56
:105C48003B434F6A3B434F6943EA87433343CE683C
:105C580033432B4323430C68234304681343636192
:105C6800B2F1406FE4D003684A689A61E0E7CB6A12
:105C78000F6B3B434F6B3B434F6A3B434F6943EAD0
:105C8800874333432B4323430C68234301681A4358
:105C98004A61CDE70D6A002D37D003688C68DC6156
:105CA800CD69E5B1CB6A0C6B23434C6B23434C6A3B
:105CB80023434C6943EA84430C6923430C6A234316
:105CC800CC6823432B438C692343046813436361E3
:105CD800B2F1406FACD003684A689A61A8E7CC6A11
:105CE8000B6B1C434B6B1C434B6A1C434B6944EACC
:105CF80083440B691C430B6A1C4345EA04038C6903
:105D0800234301681A434A6192E7CE69CEB10B6B0F
:105D1800CF6A3B434F6B3B434F6A3B434F6943EA70
:105D280087432B43CD682B433343234304681343F2
:105D38006361B2F1406F3FF47BAF03684A689A61D0
:105D480076E7D1F824C0BCF1000F3FF471AFCB6AFD
:105D58000F6B3B434F6B3B434CEA03074B6947EAE6
:105D680083431D4346EA0503234301681A434A61F6
:105D78005EE72DE9F84305460F4616469946DDF8D5
:105D880020802C68A4683C4214BF4FF0010C4FF0EF
:105D9800000CB44514D0B8F1FF3FF2D0FFF7DEFE97
:105DA800A0EB0900404502D8B8F1000FE9D104235F
:105DB80085F841306B6C43F001036B64012000E00F
:105DC8000020BDE8F8832DE9F04182B004460F4673
:105DD8001646FFF7C3FE94F840C05FFA8CFCBCF18E
:105DE800010F3CD00546012384F8403094F841C0A7
:105DF8005FFA8CFC9C4508D04FF00208002384F819
:105E08004030404602B0BDE8F081002262640223BF
:105E180084F841300096034620212046FFF7A9FF69
:105E280080460028EAD1002239462046FFF7B6FE10
:105E38007B6A1BB1012384F84130DFE700962B46CB
:105E4800012202212046FFF794FF80460028D5D181
:105E580023680222DA60012384F84130CEE74FF04C
:105E68000208CEE72DE9F04383B004468946174679
:105E7800FFF774FED4F8008094F84030DBB2012BB1
:105E880057D00646012384F8403094F84150EDB2CB
:105E98009D4207D00225002384F84030284603B0ED
:105EA800BDE8F08300236364B9F1000F3CD01223EE
:105EB80084F84130D8F810300133E362D8F8103054
:105EC8000133A362C4F82490D8F8143023F0406357
:105ED800C8F814300025E36A9BB1009733460122C5
:105EE80004212046FFF745FF054650B9636A1B7831
:105EF80088F82030616A01316162E16A0139E16242
:105F0800E9E71DB1012384F84130C4E7009733461F
:105F1800012202212046FFF72CFF05460028F1D177
:105F280023680222DA60EDE7636C43F008036364D8
:105F3800B1E70225B2E72DE9F04383B0044689466C
:105F48001746FFF70BFED4F80080D8F8182094F80D
:105F58004030DBB2012B5BD00646012384F8403089
:105F680094F84150EDB29D4207D00225002384F8F1
:105F78004030284603B0BDE8F08300236364B9F1DC
:105F8800000F40D0222384F84130D8F81030013374
:105F9800A363D8F8103001336363C4F83090D8F89D
:105FA800143023F0406343F08063C8F8143023684A
:105FB8009A610025A36B9BB1009733460122062105
:105FC8002046FFF7D6FE054650B9236B98F82020E7
:105FD8001A70216B01312163A16B0139A163E9E7D3
:105FE8001DB1012384F84130C0E7009733460122F0
:105FF80002212046FFF7BDFE05460028F1D123689F
:106008000222DA60EDE7636C43F008036364ADE7EE
:106018000225AEE7F0B583B004460E461546FFF7F5
:106028009DFD94F840C05FFA8CFCBCF1010F46D08E
:10603800012384F8403094F84120D2B29A4206D025
:10604800002384F840300227384603B0F0BD002210
:106058006264422384F84130A36C009303462021F4
:106068002046FFF786FE074618B1002384F8403023
:10607800EAE723682A689A6223686A685A6223688A
:10608800AA68DA6221680B6823F440032A69686900
:10609800024313430B6023680922DA60EB68B3629A
:1060A8004FF0006231462046FFF778FD002384F860
:1060B80040302268136843F410231360C4E70227B2
:1060C800C2E7F0B583B004460E461546FFF746FD15
:1060D80094F840C05FFA8CFCBCF1010F3BD001235F
:1060E80084F8403094F841C05FFA8CFC9C4506D097
:1060F8000227002384F84030384603B0F0BD002260
:106108006264822384F84130A36C00930346202103
:106118002046FFF72EFE07460028EAD122681368BA
:1061280023F0080369680B4313606B68082B06D0DB
:106138004FF0406231462046FFF730FDD9E723682B
:106148002A681A6323681022DA602268136843F405
:1061580080131360ECE70227CEE7704708B5006CA0
:1061680000238363C36290F84130DBB2082B0DD162
:1061780003680222DA600268136843F4003313608C
:106188000268136843F00203136008BD012380F816
:106198004130FFF7E2FFF8E77047704770477047F4
:1061A800704770477047000010B5044603689A6846
:1061B800196812F0040F3FD011F4802F3CD090F8EA
:1061C8004120D2B2122A12D090F84120D2B2222A0B
:1061D8001FD02046FFF7E4FF10BD626A127883F8EB
:1061E8002020626A01326262E26A013AE26222684F
:1061F800916811F0040FECD0E16A0029EDD1136821
:1062080023F480231360E4E7136823F480231360E6
:10621800DFE72268916811F0040FDAD0A16B00293A
:10622800F2D0226B93F820101170226B0132226396
:10623800A26B013AA263ECE712F0020F76D011F4D8
:10624800003F73D00222DA602268136823F4E02347
:10625800136094F84130DBB2122B1DD094F8413012
:10626800DBB2222B2ED094F84130DBB2022B52D075
:1062780094F84130DBB2082BAED12268536923F081
:1062880040635361012384F84130636C002B49D18A
:106298002046FFF781FF9FE723681A6812F0040F72
:1062A80009D01A6822F004021A60E36B1A68D368EE
:1062B80023F00103D360012384F841302046FFF71F
:1062C8006EFF89E721680B6813F0040F10D00B6884
:1062D80023F004030B60E36B1A68D36823F001030F
:1062E800D360012384F841302046FFF757FF73E756
:1062F80023689B6813F47C5FF3D0A36B002BF0D06A
:10630800236B91F820201A70236B01332363A36B4E
:10631800013BA363ECE7012384F841302046FFF7F3
:106328003CFF59E72046FFF718FF55E712F0080F22
:1063380014D011F4002F11D00822DA6023681A68EB
:1063480012F4800F06D01A6822F410221A60012372
:1063580084F841302046FFF724FF3DE712F0010F93
:1063680031D011F4803F2ED00122DA602268136800
:1063780023F470231360636C43F00203636423689F
:106388001A6812F0040F17D01A6822F004021A6073
:10639800E36B144A9A65E06BFFF796FA00283FF41E
:1063A8001BAF636C43F004036364012384F841303A
:1063B8002046FFF7D2FE0FE7012384F8413020463C
:1063C800FFF7CBFE08E712F0100F3FF405AF11F40A
:1063D800801F3FF401AF1022DA602046FFF7E2FE8B
:1063E800FAE600BF656100088164704770B582B045
:1063F8000446FFF7B3FB002C45D0064694F841301D
:10640800002B37D025682A6822F47062A168013908
:1064180042EA01222A60A36C00933346002220211D
:106428002046FFF7A6FC18BB21680B68174A1A40DC
:106438006568E36843EA0563E5692B43256A2B43EE
:1064480013430B6021684A68114B13402569626940
:1064580042EA0542A5692A4313434B602268136840
:1064680043F00103136000236364012384F841307F
:1064780002B070BD2046FAF76DF941F28831204626
:10648800FFF7B2FFBEE70120F2E700BF2FFFFF00D2
:10649800FEF8E0FF0268136823F490731360026843
:1064A8009168044B0B4093602023C0F8843000238C
:1064B800C3667047FEFFFFEF704708B501680A68BA
:1064C80022F040020A602022C0F8802000220267E1
:1064D800FFF7F2FF08BD704770B504460168CB6945
:1064E8000D68886840F60F021A4008D113F0200F93
:1064F80005D015F0200F30D110F0805F2DD12AB1D2
:106508006D4A02402FD16D4E35422CD113F4801FB5
:1065180003D010F4800F40F0B48013F0800F07D040
:1065280015F0800F40F0B48010F4000F40F0B080F8
:1065380013F0400F03D015F0400F40F0B08013F473
:10654800000F03D015F0804F40F0AD8013F0807F2E
:1065580002D0002DC0F2AB8070BDE36E002BFBD0E3
:1065680020469847F8E713F0010F09D015F4807F0B
:1065780006D001260E62D4F888103143C4F888107A
:1065880013F0020F0BD010F0010F08D0216802267B
:106598000E62D4F8881041F00401C4F8881013F092
:1065A800040F0BD010F0010F08D0216804260E62EA
:1065B800D4F8881041F00201C4F8881013F0080FCD
:1065C8000BD015F0200F00D13AB1226808211162D2
:1065D800D4F888200A43C4F8882013F4006F0CD03C
:1065E80015F0806F09D022684FF400611162D4F869
:1065F800882042F02002C4F88820D4F88820002A95
:10660800AAD013F0200F09D015F0200F02D110F0F6
:10661800805F03D0E36E0BB120469847D4F88820FA
:1066280023689B6813F0400F02D112F0280F21D085
:106638002046FFF72FFF23689A6812F0400F15D005
:106648009A6822F040029A60A36F5BB11C4A1A65EF
:10665800A06FFFF701F800283FF47EAFA06F036D2D
:10666800984779E72046FFF736FF75E72046FFF79A
:1066780032FF71E72046FFF72EFF0023C4F8883069
:106688006AE74FF480130B62204600F0EFFC63E7E3
:10669800236F002B3FF460AF204698475CE7204605
:1066A800FFF70BFF58E7204600F0E2FC54E72046CE
:1066B80000F0DDFC50E700BF0100001020010004DD
:1066C800CD66000808B5806B0023A0F85E30A0F8FE
:1066D8005630FFF700FF08BD70B586B00446016864
:1066E80083680269134342691343C2691343426EC4
:1066F80013430868884A02401A430A6022685368AC
:1067080023F44053E1680B435360A1692268834B2B
:106718009A4201D0236A19439068814B03400B4386
:1067280093602268D36A23F00F03616A0B43D36234
:1067380022687C4B9A4221D07B4B9A4200F08C8095
:106748007A4B9A4200F0A280794B9A4200F0B580C9
:10675800784B9A4200F0C880774B9A4200F0F48058
:10676800764B9A4200F01981754B9A4200F02C81C1
:106778006A4B9A4200F03F81802333E0714B5B6D96
:1067880003F03803282B65D8DFE813F029006400EC
:106798006400640064006400640064004D016400E7
:1067A8006400640064006400640064002B006400FA
:1067B8006400640064006400640064005E006400B7
:1067C80064006400640064006400640060006400A5
:1067D80064006400640064006400640062000123D3
:1067E80000E008234D498A4200F02F81E069B0F5A6
:1067F800004F00F0AF81202B00F20782202B00F21F
:106808005182DFE813F01E0224024F024F022702D2
:106818004F024F024F022C024F024F024F024F020B
:106828004F024F024F0231024F024F024F024F02F6
:106838004F024F024F024F024F024F024F024F02C8
:106848004F024F024F023D021023CBE72023C9E736
:106858004023C7E78023C5E73A4B5B6D03F0070386
:10686800052B11D8DFE813F00600E10008000A0044
:106878000C000E000023B5E70823B3E71023B1E7A7
:106888002023AFE74023ADE78023ABE72D4B5B6DBB
:1068980003F00703052B0ED8DFE803F003C905074B
:1068A800090B00239EE708239CE710239AE720237F
:1068B80098E7402396E7802394E7224B5B6D03F02B
:1068C8000703052B0ED8DFE803F003B40507090B0F
:1068D800002387E7082385E7102383E7202381E740
:1068E80040237FE780237DE7164B5B6D03F00703AA
:1068F800052B0ED8DFE803F0039F0507090B0023DB
:1069080070E708236EE710236CE720236AE740232B
:1069180068E7802366E700BFF369FFCF000C0058E3
:10692800FFF4FF11001001400044004000480040FF
:10693800004C004000500040001401400078004026
:10694800007C0040004402587D4B5B6D03F0380327
:10695800282B20D8DFE803F0151F1F1F1F1F1F1F3C
:10696800711F1F1F1F1F1F1F171F1F1F1F1F1F1FE5
:10697800191F1F1F1F1F1F1F1B1F1F1F1F1F1F1F29
:106988001D0001232EE708232CE710232AE72023E4
:1069980028E7402326E7802324E7694B5B6D03F053
:1069A8000703052B0ED8DFE803F0034A0507090B98
:1069B800002317E7082315E7102313E7202311E71F
:1069C80040230FE780230DE75D4B5B6D03F0070362
:1069D800052B0ED8DFE803F003350507090B002364
:1069E80000E70823FEE61023FCE62023FAE640230E
:1069F800F8E68023F6E603F50E339B6D03F00703F4
:106A0800052B0ED8DFE803F0031F0507090B022347
:106A1800E8E60823E6E61023E4E62023E2E640233E
:106A2800E0E68023DEE60423DCE60423DAE604233A
:106A3800D8E60423D6E60423D4E60423D2E60423C6
:106A4800D0E60423CEE60423CCE6202B27D8022B5D
:106A5800C0F01A81023B1E2B00F21881DFE813F008
:106A68005000160156001601160116015B001601AA
:106A7800160116011601160116011601600016010D
:106A88001601160116011601160116011601160146
:106A98001601160116011601160116016C00402B8D
:106AA8002CD14FF40040626A264B33F81220B0FB19
:106AB800F2F3656805EB4501994200F2E980B3EB12
:106AC800053F00F2E780002633463146F9F7E0FB40
:106AD800090241EA106100026B08C0182A463346D1
:106AE80041F10001F9F7D4FBA0F54072164B9A4228
:106AF80000F2D2802368D8603046D4E00120D2E08A
:106B0800FEF7E8F90028CED10020CCE003A8FEF774
:106B1800F3F90498F6E76846FEF7EAFA0198F1E710
:106B2800074B1B6813F0200F08D0054B1B68C3F3F5
:106B3800C1030648D840E5E70548B4E70348B2E78B
:106B48000044025868890008FFFC0F000090D00339
:106B580000093D00202B15D8202B00F29F80DFE88C
:106B680003F031379D9D3A9D9D9D3F9D9D9D9D9D27
:106B78009D9D449D9D9D9D9D9D9D9D9D9D9D9D9D96
:106B88009D9D5000402B1BD1626A4D4B33F812304B
:106B9800B0FBF3F06268530803EB4000B0FBF2F07F
:106BA80080B2A0F110024FF6EF739A4278D820F025
:106BB8000F03C0F3420018432368D860002072E036
:106BC800012070E0FDF782FB0028DDD100206AE09B
:106BD800FDF78EFBF8E703A8FEF78EF90498F3E7B4
:106BE8006846FEF785FA0198EEE7364B1B6813F006
:106BF800200F08D0334B1B68C3F3C1033248D84079
:106C0800E2E73248C0E73048BEE7402B17D14FF4DF
:106C18000040626A2A4B33F81230B0FBF3F0636825
:106C280000EB5300B0FBF3F080B2A0F110024FF676
:106C3800EF739A4241D82368D860002033E00120DE
:106C480031E0FDF743FB0028E3D100202BE0FDF7FE
:106C58004FFBF8E703A8FEF74FF90498F3E76846F7
:106C6800FEF746FA0198EEE7164B1B6813F0200F63
:106C780008D0144B1B68C3F3C1031348D840E2E79C
:106C88001248C6E71048C4E701200CE001200AE0DA
:106C9800012008E0012006E0012004E0012002E0D4
:106CA800012000E001200123A4F86A30A4F868302C
:106CB8000023E366236706B070BD0120F3E700BF39
:106CC80068890008004402580090D00300093D007C
:106CD800836A13F0010F06D00268536823F4003367
:106CE800C16A0B435360836A13F0020F06D002682F
:106CF800536823F48033016B0B435360836A13F0AA
:106D0800040F06D00268536823F48023416B0B43B9
:106D18005360836A13F0080F06D00268536823F49F
:106D28000043816B0B435360836A13F0100F06D046
:106D38000268936823F48053C16B0B439360836AA2
:106D480013F0200F06D00268936823F40053016CF7
:106D58000B439360836A13F0400F0AD002685368AC
:106D680023F48013416C0B435360436CB3F5801FCD
:106D78000BD0836A13F0800F06D00268536823F49F
:106D88000023C16C0B43536070470268536823F4B7
:106D9800C003816C0B435360EBE72DE9F8430546CC
:106DA8000F4616469946DDF820802C68E46937EAD4
:106DB80004030CBF4FF0010C4FF0000CB44541D157
:106DC800B8F1FF3FF1D0FEF7C9FEA0EB090040453E
:106DD80024D8B8F1000F21D02B681A6812F0040FDC
:106DE800E3D0DA6912F4006FDFD04FF400621A6260
:106DF8002A68136823F4D07313602A68936823F011
:106E0800010393602023C5F88030C5F88430C5F8A5
:106E18008830002385F87C30032014E02A68136842
:106E280023F4D07313602A68936823F001039360F6
:106E38002023C5F88030C5F88430002385F87C30DD
:106E4800032000E00020BDE8F8832DE9F04182B07E
:106E58001E46D0F88030202B58D104460D46904667
:106E6800002A18BF002955D090F87C30012B53D048
:106E7800012380F87C300023C0F888302123C0F833
:106E88008030FEF76BFE0746A4F85480A4F85680BD
:106E9800A368B3F5805F05D04FF00008002384F89D
:106EA8007C3012E0236913B14FF00008F6E7A846DA
:106EB8000025F3E715F8012B23689A62B4F85620E9
:106EC80092B2013A92B2A4F85620B4F856309BB266
:106ED80083B100963B46002280212046FFF75DFFE4
:106EE800E0B9002DE6D138F8023B2268C3F3080365
:106EF8009362E3E700963B46002240212046FFF7D5
:106F08004CFF68B92023C4F8803000E0022002B0AA
:106F1800BDE8F0810120FAE70220F8E70320F6E750
:106F28000320F4E730B583B004460023C0F8883066
:106F3800FEF714FE05462268126812F0080F0ED1FB
:106F480023681B6813F0040F17D12023C4F880307E
:106F5800C4F88430002084F87C0003B030BD6FF0A2
:106F68007E430093034600224FF400112046FFF7AA
:106F780014FF0028E4D00320EFE76FF07E4300936E
:106F88002B4600224FF480012046FFF706FF002819
:106F9800DBD00320E1E778B310B50446D0F88030A1
:106FA8000BB32423C4F880302268136823F001034C
:106FB80013602046FFF790FB012813D0A36ABBB9E2
:106FC8002268536823F4904353602268936823F03F
:106FD8002A0393602268136843F001031360204674
:106FE800FFF7A0FF10BD80F87C30F9F731FCD8E737
:106FF8002046FFF76DFEE3E70120704784B00346A3
:10700800184A92E8030004AA02E9030016496A46EE
:1070180003C982E803005A6E32B90122A3F86A2034
:10702800A3F8682004B0704719688A68C2F34262FE
:10703800886804A901EB507010F8081C090110F8C1
:10704800100C91FBF0F1A3F86A1004A90A4412F895
:10705800081C090112F8102C91FBF2F2A3F8682021
:10706800E0E700BF60870008808900087047704724
:10707800704790F87C30012B18D0012380F87C30C1
:107088002423C0F8803003681A68196821F00101C8
:10709800196022F000520023436601680A6020222A
:1070A800C0F8802080F87C3018467047022070476E
:1070B80038B590F87C30012B1DD00446012380F8A8
:1070C8007C302423C0F8803003681D681A6822F0D9
:1070D80001021A600268936823F0604319439160C3
:1070E800FFF78CFF23681D602023C4F88030002040
:1070F80084F87C0038BD0220FCE738B590F87C3075
:10710800012B1DD00446012380F87C302423C0F8CD
:10711800803003681D681A6822F001021A6002684C
:10712800936823F0606319439160FFF767FF236852
:107138001D602023C4F88030002084F87C0038BD0E
:107148000220FCE7184AD2F8883043F47003C2F8EA
:107158008830164B1A6842F001021A6000221A6140
:1071680018681349014019609A61DA611A629A62D3
:10717800DA621A635A639A63DA631A645A6419689A
:1071880021F4802119601A660A4B1A680A4B1340C9
:10719800B3F1005F03D2094B0122C3F80821024B67
:1071A8004FF000629A60704700ED00E0004402581A
:1071B8007FEDF6EA0010005C0000FFFF0080005140
:1071C800C0B108B50346D0F8B80210B10020C3F822
:1071D800B802D3F8CC0210B10020C3F8CC0209B130
:1071E800C3F8B412012183F89C121A701846FAF7F2
:1071F80059FF08BD0320704710B582B00023ADF8D1
:10720800063059B10446C0F8B8128B6A0DF1060071
:107218009847C4F8CC02002002B010BD0320FBE759
:1072280008B5FAF796FF08BD10B50446D0F8B8328D
:1072380013B15B6801799847D4F8CC3213B10023B5
:10724800C4F8CC322046FAF78CFF10BD08B5D0F848
:10725800B83213B11B68984708BD0320FCE708B58E
:10726800D0F8B8320BB15B689847002008BD38B534
:10727800044600F2AA25284600F02EF90123C4F896
:107288009432B4F8B032C4F8983294F8AA1201F0E3
:107298001F03012B0DD0022B10D02BB101F0800160
:1072A8002046FAF771FF03E02946204600F0D6FA97
:1072B80038BD2946204600F009FBF9E72946204653
:1072C80000F038FBF4E738B504460D4631BB1346E9
:1072D800D0F89422032A01D0084638BDD0F85C11B2
:1072E800D0F8602191420CD8D0F8B8321B691BB194
:1072F80090F89C22032A0FD0204600F059FC28461B
:10730800EBE7891AC0F85C118A4228BF0A46194679
:1073180000F046FC2846E0E79847EDE7D0F8B83299
:107328009B692BB190F89C22032A03D19847D4E794
:107338000320D2E70320D0E738B504460D460029DC
:1073480048D11346D0F89422022A05D094F8A032E6
:10735800012B3AD0284638BDC269016A8A4211D841
:107368008A421BD0D4F8B832DB681BB194F89C224F
:10737800032A27D080212046FAF706FF204600F08E
:1073880022FCE3E7521AC261194600F0F2FB00231F
:107398001A4619462046FAF717FFD7E78369994234
:1073A800E0D8D0F898229342DCD20022114600F0AF
:1073B800E0FB0021C4F898120B460A462046FAF76B
:1073C80003FFC3E720469847D4E7002384F8A03298
:1073D8002846C0E7D0F8B8325B692BB190F89C22F8
:1073E800032A03D19847B6E70320B4E70320B2E79E
:1073F80070B50446012380F89C320023C0F894320B
:107408004360C0F8A432D0F8BC3223B1D0F8B83207
:107418005B68002198474023002211462046FAF76E
:10742800A8FE0126A4F864614025C4F860512B46E3
:10743800002280212046FAF79CFEA68425620020BF
:1074480070BD01740020704790F89C3280F89D321E
:10745800042380F89C320020704790F89C32042B5B
:1074680001D00020704790F89D3280F89C32F8E7F0
:1074780008B590F89C32032B01D0002008BDD0F845
:10748800B832DB69002BF8D09847F6E70020704740
:10749800002070470020704708B5012380F89C320F
:1074A800D0F8B83213B15B6801799847002008BD5D
:1074B8000346002002E00130C0B201331A78002AE6
:1074C800F9D1704708B54B88012B00D008BDC0F82A
:1074D800A43200F06DFBF9E70B7803704B7843702A
:1074E8008B78CA7843EA022343800B794A7943EAC6
:1074F800022383808B79CA7943EA0223C3807047C9
:1075080010B504468021FAF73FFE00212046FAF71D
:107518003BFE10BD30B583B004460D460023ADF8E0
:10752800063049880B0A013B062B00F2B380DFE8DE
:1075380003F0041F33B1B195A200D0F8B4321B6830
:107548000DF10601007C9847EA88002A00F0AB801C
:10755800BDF80630002B00F0A1809A4228BF1A46D9
:10756800ADF806200146204600F0F6FA03B030BD1B
:10757800037C43B9D0F8B8329B6A0DF106009847EE
:1075880002234370E0E7D0F8B832DB6A0DF1060059
:10759800984702234370D7E7C9B2052952D8DFE8D4
:1075A80001F003101D2A3744D0F8B4325B6823B1C8
:1075B8000DF10601007C9847C6E72946FFF7A0FFB2
:1075C800D4E7D0F8B4329B6823B10DF10601007CF2
:1075D8009847B9E72946FFF793FFC7E7D0F8B432D1
:1075E800DB6823B10DF10601007C9847ACE729461A
:1075F800FFF786FFBAE7D0F8B4321B6923B10DF163
:107608000601007C98479FE72946FFF779FFADE719
:10761800D0F8B4325B6923B10DF10601007C9847BC
:1076280092E72946FFF76CFFA0E7D0F8B4329B69D0
:1076380023B10DF10601007C984785E72946FFF73D
:107648005FFF93E7D0F8B8329B6B1BB10DF10602D0
:10765800984779E72946FFF753FF87E7037C33B953
:10766800D0F8B8325B6B0DF1060098476CE72946F5
:10767800FFF746FF7AE7037C43B9D0F8B8321B6BB3
:107688000DF106009847072343705DE72946FFF789
:1076980037FF6BE72946FFF733FF67E729462046A0
:1076A800FFF72EFF62E7204600F082FA5EE738B562
:1076B80004468B88F3B9CB88E3B94B887F2B19D85C
:1076C80003F07F0590F89C32032B0CD080F89E5273
:1076D8002946FAF769FD204600F06AFA35B1022317
:1076E80084F89C3209E0FFF70BFF06E0012384F8D9
:1076F8009C3202E02046FFF703FF38BD70B5044610
:107708000E468D782D4B1D70012D0FD890F89C32A8
:10771800022B0FD0032B23D0FFF7F2FE274B19784B
:107728002046FFF79CFD0325284670BDFFF7E8FEBD
:107738000325F9E78DB145602946FFF787FD054622
:1077480020B131462046FFF7DBFEEDE7204600F08A
:107758002FFA032384F89C32E6E700F029FAE3E7DE
:10776800CDB141688D4225D0C9B2FFF778FD134BE2
:10777800197861602046FFF769FD0546B0B13146CA
:107788002046FFF7BDFE21792046FFF768FD02235A
:1077980084F89C32C8E7022380F89C324560294669
:1077A800FFF75DFD204600F003FABDE7204600F034
:1077B800FFF9B9E700F0FCF90025B5E7440B002014
:1077C80008B5CB88012B0AD190F89C32022B09D935
:1077D800032B09D10122011D00F0BEF901E0FFF7DA
:1077E8008FFE08BD5BB213B9FFF78AFEF9E70146C1
:1077F800002341F8083F012200F0AEF9F1E708B58F
:1078080090F89C32013B022B12D8CB88022B0CD16A
:107818000123C360D0F8A4320BB10323C360022252
:1078280000F10C0100F098F908BDFFF769FEFBE7CD
:10783800FFF766FEF8E708B590F89C32013B022B8B
:1078480009D84B88012B00D008BD0023C0F8A4320A
:1078580000F0AEF9F8E7FFF753FEF5E738B50C7816
:1078680004F06004202C06D0402C04D054B1FFF75B
:1078780047FE002404E0D0F8B8329B6898470446D5
:10788800204638BD4D78092D1DD8DFE805F01219BE
:107898001C161C08051C0F0BFFF73CFEF0E7FFF752
:1078A80006FFEDE7FFF72AFF0446E9E7FFF788FF41
:1078B800E6E7FFF7A4FF2C46E2E7FFF703FEDFE762
:1078C800FFF7B9FFDCE7FFF71BFED9E770B5054600
:1078D8000C460B7803F06003202B07D0402B05D013
:1078E80023B1FFF70DFE0026304670BD95F89C3297
:1078F800013B022B18D82379012B0FD8D5F8B832C1
:107908009B682146284698470646E388002BEBD11A
:107918000028E9D1284600F04BF9E5E7214628463A
:10792800FFF7EEFD0026DFE721462846FFF7E8FDD2
:107938000026D9E7F8B506460D468B880C7804F082
:107948006004202C08D0D9B2402C05D06CB129464F
:10795800FFF7D6FD002406E0D6F8B8329B68294622
:107968003046984704462046F8BD6F78012F2FD03F
:10797800032F05D0002F57D02946FFF7C1FDF2E7A6
:1079880090F89C32022B05D0032B12D02946FFF722
:10799800B7FDE8E7002918BF802906D0FAF7F4FBFD
:1079A80080213046FAF7F0FBDDE72946FFF7A8FD0E
:1079B800D9E76B882BB9002918BF802901D0EB883B
:1079C8001BB1304600F0F4F8CDE7FAF7DDFBF8E735
:1079D80090F89C32022B05D0032B12D02946FFF7D2
:1079E8008FFDC0E7002918BF802906D0FAF7CCFB25
:1079F80080213046FAF7C8FBB5E72946FFF780FD36
:107A0800B1E76B88002BAED111F07F0F09D130465A
:107A180000F0CEF8D6F8B8329B6829463046984729
:107A2800A1E7FAF7B9FBF2E790F89C22022A06D000
:107A3800032A2AD02946FFF763FD3C4693E700292D
:107A480018BF802913D113F0800F15D101F07F01E1
:107A580001EB8101890001F5A8710144043100237B
:107A68000B600222304600F077F83C467BE7294657
:107A7800FFF746FD3C4676E701F07F0101EB810107
:107A88008900103101440431E9E75BB2002B20DBA7
:107A980001F00F0202EB820200EB8202B2F86421CD
:107AA8002AB3002B28DB01F07F0303EB83039C0040
:107AB80004F5A87434440434802918BF002924D15B
:107AC8000023236002222146304600F045F83C4658
:107AD80049E701F00F0202EB820200EB8202928C6E
:107AE800002ADED12946FFF70BFD3C463BE7294635
:107AF800FFF706FD3C4636E701F07F0303EB8303FF
:107B08009C00103434440434D6E73046FAF700FBBE
:107B180010B101232360D5E700232360D2E7D0B159
:107B280070B50D4616460446FFF7C2FC431C5B00C1
:107B38009BB233802B7003236B70022307E0EA5457
:107B480001345A1CD2B20021A9540233DBB2227884
:107B5800002AF4D170BD704708B513460222C0F858
:107B680094228361C3610A460021FAF725FB0020AD
:107B780008BD08B513460A460021FAF71DFB002088
:107B880008BD08B513460322C0F89422C0F858313E
:107B9800C0F85C310A460021FAF716FB002008BD40
:107BA80008B513460A460021FAF70EFB002008BD67
:107BB80008B50423C0F8943200231A461946FAF788
:107BC800FBFA002008BD08B50523C0F8943200234D
:107BD8001A461946FAF7F8FA002008BD1B23038055
:107BE80000487047B8000020002070470020704708
:107BF8000A23038000487047D4000020D0F8BC3224
:107C080003F58052127E0A2A0CD003F580530A210C
:107C180019760E221A7400225A749A74DA74197535
:107C28005A75704703F580530221197600221A7499
:107C38005A749A74DA7419755A757047D0F8BC3248
:107C480003F58052117E8A1ED2B2052918BF012A77
:107C580003D9062901D009290CD103F58053022143
:107C6800197600221A745A749A74DA7419755A7546
:107C78001A605A6070470000D0F8C032062907D849
:107C880010B5044C21461868FFF749FF204610BD7F
:107C980000207047480B002008B5D0F8BC3203F527
:107CA800805200215176134A127D12F0040F09D038
:107CB80003F580530621197600225A749A74DA74EF
:107CC800197508BD03F580530821197600225A74E6
:107CD8009A74DA741975FFF7A7FABFF34F8F06493C
:107CE800CA6802F4E062054B1343CB60BFF34F8FC1
:107CF80000BFFDE7B800002000ED00E00400FA0531
:107D080030B583B0D0F8BC42D0F8C02204F5805317
:107D18001B7E042B04D0072B5ED0002003B030BD9F
:107D280004F58053196800293DD15B68012B47D0C1
:107D3800052B2AD12378212B16D0412B40D16078EE
:107D480004F580539860A17800EB01209860E178F1
:107D580000EB01409860217900EB01609860D368DE
:107D6800984768B30320D9E7637804F58052936095
:107D7800A17803EB01239360E17803EB014393605F
:107D8800217903EB016393601AE004F58053002224
:107D98005A601A608DF800200123ADF80630694654
:107DA800FFF7AEFB0CE001290AD9023904F580532C
:107DB800986815695A6800EB01312046A84778B9D8
:107DC80004F58054002060602060032323766074EB
:107DD800A074E0742375A1E7FFF75EFF00209DE71C
:107DE80003209BE770B5D0F8BC32D0F8C052CA88DF
:107DF800002A58D0044603F58052127E092A18BF7B
:107E0800022A48D1488803F5805CCCF80000CA886B
:107E1800CCF80420B8B9032A13D9022003F58052FC
:107E28001076002151749174D17410751970212243
:107E38005A7041229A70032219462046FFF78CFE99
:107E48003AE00920EAE7012818D903F580564FF0EF
:107E5800090C86F818C000217174B174F17486F8A1
:107E680014C002386D691946B36803EB0030A8479F
:107E7800014672682046FFF76FFE1DE003F5805348
:107E88000F20187600225A749A74DA7418752046EE
:107E9800FFF736FB10E003F5805300225A601A60A2
:107EA800FFF72EFB08E003F5805302211976002224
:107EB8005A749A74DA74197570BD000070B5044666
:107EC800D0F8BC52D0F8C02205F580531B7E032B96
:107ED80009D0062B36D0062241F21001294420464B
:107EE800FFF73AFE70BD05F580535B6803B305F5EF
:107EF800805304201876002159749974D974187520
:107F08001B6813B92B78412B09D0966905F5805366
:107F180041F210022A4401219868B047DBE79669CC
:107F280005F5805341F210022A449868B047D2E719
:107F380005F580530521197600225A749A74DA746B
:107F48001975C8E705F580535B7E012B10D0002B0F
:107F5800C1D10D4B1B7D13F0040FBCD005F5805328
:107F68000221197600225A749A74DA741975B2E7E4
:107F780005F5805307221A76012159740021997456
:107F8800D9741A75A7E700BFB800002008B5D0F863
:107F9800BC32012241F218011944FFF7DDFD08BD8A
:107FA80008B5D0F8BC32CA88D2B103F58052127E27
:107FB800052A18BF022A10D14A8803F5805CCCF83C
:107FC8000020CA88CCF8042003218CF818108CF8FB
:107FD80014101946FFF7D5FD14E0FFF791FA11E0E8
:107FE80003F58052127E022A18BF052A0BD103F529
:107FF800805301225A760621197600225A749A74FF
:10800800DA74197508BDFFF77BFAFBE710B504466B
:10801800D0F8BC3203F58052107E821ED2B20528F9
:1080280018BF012A03D9062801D009280CD103F565
:1080380080530220187600221A745A749A74DA74DB
:1080480018755A751A605A60074B5B7D13F0100F4C
:1080580006D02046FFF7E8F82046FFF7E1F810BD04
:108068004888FDF781FDFAE7B800002030B583B0F5
:10807800D0F8BC220023ADF806300C7814F0600468
:1080880029D0202C75D14C78062C20D8DFE804F0B4
:108098001C04080C10141800FFF782FF00246BE082
:1080A800FFF7A0FE002467E0FFF708FF002463E065
:1080B800FFF7A4FD00245FE0FFF768FF00245BE002
:1080C800FFF7BCFD002457E0FFF7A0FF54E0FFF7DF
:1080D80017FA032450E04D780B2D46D8DFE805F059
:1080E800064C4545454515454545243390F89C3291
:1080F800032B03D0FFF704FA03243DE002220DF11D
:108108000601FFF729FD2C4636E04B881B0A212B78
:1081180004D000221146FFF71FFD2DE0CA88092A66
:1081280028BF09221649F6E790F89C32032B03D0A2
:10813800FFF7E6F903241FE002F580530122D9680E
:10814800FFF70AFD18E08C785CB990F89C32032B95
:1081580003D102F58052D4600EE0FFF7D1F9032471
:108168000AE0FFF7CDF9032406E0FFF7C9F9032475
:1081780002E0FFF7C5F90324204603B030BD00BF75
:10818800CA00002038B5D0F8BC32ABB1054603F5BB
:10819800805300241C605C6002221A761C741A75D5
:1081A800D0F8C0329B689847D5F8BC0200F08CF82C
:1081B800C5F8BC42204638BD0220FCE710B504468D
:1081C80041F21C0000F078F8C8B1C4F8BC0200F510
:1081D80080530022DA604FF0104199601A605A60AB
:1081E8005A76022119761A745A749A74DA741975BF
:1081F8005A75D4F8C0325B68984728B910BD002377
:10820800C4F8BC320220F9E70320F7E719B1C0F837
:10821800C01200207047032070470000DFF834D0F8
:10822800FEF790FF002103E00B4B5B5843500431ED
:108238000A480B4B42189A42F6D30A4A02E0002336
:1082480042F8043B084B9A42F9D300F011F8F8F7CA
:108258007BF9704700000220AC890008000000206C
:108268004401002044010020640C0020FEE70000C7
:1082780070B50D4D0D4C641BA4100026A64209D103
:108288000B4D0C4C00F05CFA641BA4100026A642AF
:1082980005D170BD55F8043B98470136EEE755F80F
:1082A800043B98470136F2E7A4890008A48900082E
:1082B800A4890008A8890008024B0146186800F044
:1082C80063B800BFE0000020024B0146186800F0C8
:1082D8000BB800BFE000002002440346934200D1DF
:1082E800704703F8011BF9E737B5002948D051F862
:1082F800043C0190002BA1F10404B8BFE41800F07D
:10830800AFF8204A01981368154633B963601460C2
:1083180003B0BDE8304000F0A9B8A3420BD92168EA
:108328006218934204BF1A685B68636004BF5218FE
:1083380022602C60ECE71A465B680BB1A342FAD9BD
:1083480011685518A5420BD1246821445418A3423A
:108358001160DDD11C685B68536021441160D7E768
:1083680002D90C230360D3E7256861198B4204BF47
:1083780019685B68636004BF491921605460C7E7E6
:1083880003B030BD480C0020F8B5CD1C25F003051E
:1083980008350C2D38BF0C25002D064601DBA942F7
:1083A80003D90C2333600020F8BD00F059F82149A7
:1083B8000A6814469CB9204F3B6823B921463046C9
:1083C80000F03CF838602946304600F037F8431C86
:1083D80023D10C233360304600F048F8E3E72368E4
:1083E8005B1B17D40B2B03D923601C44256004E0C6
:1083F8006368A2420CBF0B605360304600F036F849
:1084080004F10B00231D20F00700C21ACCD01B1A60
:10841800A350C9E722466468CCE7C41C24F00304CF
:10842800A042E3D0211A304600F008F80130DDD12F
:10843800CFE700BF480C00204C0C002038B5064D93
:108448000023044608462B6000F016F8431C02D1AE
:108458002B6803B1236038BD600C0020704770475B
:108468000148FFF7FBBF00BF580C00200148FFF789
:10847800F6BF00BF580C0020044A05491368002BBA
:1084880008BF0B461844106018467047500C00206F
:10849800680C00202DE9F04F099E88468E46154647
:1084A80004461946002B40F0C7804245B2FA82F7CD
:1084B80046D94FB1C7F1200C08FA07F320FA0CFC93
:1084C800BD404CEA030EBC404FEA15481FFA85FC34
:1084D800BEFBF8F9220C08FB19E309FB0CFA42EA87
:1084E80003439A4528D9EB1809F1FF3004D29A457D
:1084F80002D9A9F102002B44A3EB0A03A4B2B3FBEF
:10850800F8F208FB123302FB0CFC44EA0344A445CE
:1085180014D92C1902F1FF3303D2A44501D9931EB3
:108528002C44A4EB0C0443EA00401EB1FC40002399
:1085380034607360BDE8F08F4846DDE71346F0E726
:1085480002B9FFDE8FBBA8EB020301214FEA154EEB
:10855800AAB2B3FBFEFC200C0EFB1C330CFB02F88A
:1085680040EA0343984563D9EB180CF1FF3004D275
:10857800984502D9ACF102002B44A3EB0803A4B23E
:10858800B3FBFEFC0EFB1C330CFB02F244EA034473
:10859800A2424FD92C190CF1FF3304D2A24202D9BE
:1085A800ACF102032C44A41ABDE7C7F1200C28FA49
:1085B8000CF908FA07F320FA0CFCBD404CEA030258
:1085C8004FEA154EABB2B9FBFEFC110C0EFB1C902A
:1085D8000CFB03F841EA0040804504FA07F423D96C
:1085E80028180CF1FF3104D2804502D9ACF1020100
:1085F8002844A0EB080092B2B0FBFEFC0EFB1C0066
:108608000CFB03F842EA004398450FD9EB180CF12C
:10861800FF3204D2984502D9ACF102022B44A3EBF5
:10862800080342EA014191E76146E2E76246F6E75C
:108638006046A2E76346B6E7434505D90EB1C6E9E9
:1086480000080021084675E7B3FA83FCBCF1000F67
:1086580010D1434501D382420AD8841A68EB030338
:1086680001209E46002E68D0C6E9004E002161E731
:108678006046F7E7CCF1200E03FA0CF322FA0EF469
:108688001C4320FA0EF108FA0CF328FA0EFB1943E2
:108698004FEA144902FA0CF5BBFBF9F8A3B209FB3F
:1086A80018BB0A0C08FB03FA42EA0B42924500FA8F
:1086B8000CF73ED9A21808F1FF3004D2924502D92E
:1086C800A8F102002244A2EB0A0289B2B2FBF9F82F
:1086D80009FB182208FB03F341EA024293422AD914
:1086E800A21808F1FF3104D2934202D9A8F102017D
:1086F800224441EA0040A0FB0598D21A42454B4665
:10870800414602D306D14F4504D2B9EB050368EBC5
:10871800040101388EB1FC1A62EB010707FA0EFE5C
:1087280024FA0CF34EEA030327FA0CF7C6E90037DC
:108738009CE74046C7E74146DBE73146FAE60000DA
:10874800F8B500BFF8BC08BC9E467047F8B500BF36
:08875800F8BC08BC9E46704706
:1087600001010103070100004D61696E3A204D6669
:10877000673A20307825780D0A000000515350499F
:10878000206D6170706564206F6B210D0A00000020
:1087900056616C696420535020666F756E64210DBC
:1087A0000A000000456E7472793A2030782530381E
:1087B0006C780D0A000000004E6F2076616C6964D1
:1087C00020696D61676520666F756E64210D0A0012
:1087D000666E6900666E692B000000006E616E00B7
:1087E000666E692D00000000000000000000F03FF0
:1087F000000000000000244000000000000059407C
:108800000000000000408F40000000000088C340CE
:1088100000000000006AF8400000000080842E4143
:1088200000000000D01263410000000084D797418F
:108830000000000065CDCD4153544D333220446FCC
:10884000776E4C6F6164204669726D776172652046
:10885000557064617465000053544D6963726F65AF
:108860006C656374726F6E696373000044465520D3
:10887000436F6E666967000044465520496E746513
:1088800072666163650000004D656D5F49665F5209
:108890006561645F46533A204164643A203078252C
:1088A0003038780D0A0000004D656D5F49665F57EE
:1088B000726974655F46533A204164643A203078A7
:1088C00025303878205372633A2030782530387854
:1088D000204C656E3A20307825303878203153743A
:1088E0003A203078253032780D0A00004D656D5FF2
:1088F00049665F57726974655F46533A20506765F1
:108900003A203078253038780D0A00004D656D5FCB
:1089100049665F45726173655F46533A20416464FE
:108920003A203078253038780D0A00004D454D5FEB
:1089300049665F496E69745F46533A204D66673AEF
:1089400020307825780D0A00405153504920466C5C
:108950006173682F307839303030303030302F3418
:108960003039362A344B670001000200040006004B
:1089700008000A000C0010002000400080000001E8
:1089800008040204080101010000000000000000CA
:0C899000010203040102030406070809A9
:08899C0000FBFF7F0100000059
:0489A400F1020008D4
:0489A800CD020008F4
:1089AC00C11C0008CD1C0008911D00086D1D00089D
:1089BC00591D0008AD1D0008D11D00081201000250
:1089CC0000000040830411DF0002010203010000DB
:1089DC00040309041A03000000000000000000005A
:1089EC00000000000000000000000000000000007B
:1089FC0048890008ED1E0008F51D0008C91E000876
:108A0C00511E0008191E0008F91D00080100000085
:108A1C00100000000090D0030090D003C581000826
:108A2C008D81000875800008097D0008F17B000825
:108A3C000000000000000000F57B000800000000B2
:108A4C0000000000E57B0008E57B0008E57B0008E2
:108A5C00F97B0008817C000809021B00010102C09F
:108A6C00320904000000FE01020609210BFF000080
:108A7C00101A01000A06000200000040010000006C
:108A8C00E4000020000000000000000000000000D6
:108A9C0000000000000000000000000000000000CA
:108AAC0000000000000000000000000000000000BA
:108ABC0000000000000000000000000000000000AA
:108ACC00000000000000000000000000000000009A
:108ADC00000000000000000000000000000000008A
:048AEC000000000086
:040000050800822548
:00000001FF
